:1066D800011300000501013C0200000301FA040057
:1066E800FA0500030A0A5A0B001E0C00FA0D0003F3
:1066F8000E00030F0164100096120132130AFA14F7
:10670800010215000217010A1801FA1905321A01C7
:106718000A1B01FA1C05321FFFFF20FFFF23011E81
:106728002400642A00FA2B00FA2C50782D003D2E04
:1067380000462F001E3000643250783432FA35019A
:1067480064360164370150380A643C00643E003CFA
:106758003F000140FFFF411450420A5A430AC8440F
:1067680005324500B44600FA4701784802034C0058
:10677800FA4EFFFF500808510596520A32530B464D
:10678800540A96560102570546580002590A465AB5
:1067980032FA5B010A5C0A325E000A5F00FE61FFA2
:1067A800FF64021C6600026701016A0A3C6B000074
:1067B8006C32967300007400007801327901327EE1
:1067C800FFFF81FFFF84FFFF8500AF860001870080
:1067D800FA89010A8A00009900009D0A969E000124
:1067E8009FFFFFFAFAFA00000501013C02000003CE
:1067F80001FA0400FA0500030A0A5A0B001E0C00ED
:10680800FA0D00030E00030F016410009612013206
:10681800130AFA14010215000017010A1801FA19DF
:1068280005321A010A1B01FA1C05321FFFFF20FF5F
:10683800FF23011E2400642A00FA2B00FA2C50784A
:106848002D003D2E00462F001E3000643250783453
:1068580032FA350164360164370150380A643C0065
:10686800643E003C3F000140FFFF411450420A5A79
:10687800430AC84405324500B44600FA47013C487B
:1068880002024C00FA4EFFFF500808510596520AC2
:1068980032530B46540A96560101570546580001D3
:1068A800590A465A32FA5B010A5C0A325E000A5FEC
:1068B80000FE61FFFF64031C6600026701016A0AAB
:1068C8003C6B00006C329673000074000078013253
:1068D8007901327EFFFF81FFFF84FFFF85FFFF867E
:1068E800FFFF87FFFF8901028A00009900009D0AC7
:1068F800969E00019FFFFFFAFAFA0065006F007983
:106908000083008D009700A100AC00B600C000CA4B
:1069180000D400DE00E800F2005B0063006A007249
:10692800007A008200890091009900A100A800B0B7
:1069380000B800BF00C700CF00D600DF00E600EEB9
:1069480000F600400046004C00520059005F006508
:10695800006B00710077007D00830089008F00952F
:10696800009C00A200A800AE00B400BA00C000C697
:0E69780000CC00D200D900DF00E500EB00F1FA
:1035E70090005FE0D3940440149007D0E0FEA3E07E
:1035F700FF9066DA126ABFE493F59980129007D0BC
:10360700E0FEA3E0FF9067EE126ABFE493F599909E
:1036170007D0E0FEA3E0FF9066D8E493FC74019323
:10362700FDEFB50507EEB50403754D009007D01201
:103637006AA62285F97285FA737E017F00E5731207
:103647006A98E5722FFF50010E8E598F5A90001B12
:10365700E0FCA3E0FDEF2DFDEE3CFC8C5B8D5C22D6
:1036670075A71085F97285FA737E017F00E57312DD
:103677006A98E5722FFF50010E8E598F5A90001BE2
:10368700E0FCA3E0FDEF2DFDEE3CFC8C5B8D5C22A6
:10369700E55CF5FBE55BF5FCD29322E55CF5E9E536
:1036A7005BF5EAD29422E55CF5EBE55BF5ECD291AC
:1036B70022E55CF5EDE55BF5EED29222E55CF5FBE4
:1036C700E55BF5FCD28722E55CF5E9E55BF5EAD237
:1036D7009022E55CF5EBE55BF5ECE5B54410F5B557
:1036E70022E55CF5EDE55BF5EEE5B54420F5B522A1
:1036F700AE59AF5A74068E048F05FF126A888C5B29
:103707008D5CAE59AF5A74068E048F05FF126AB3EB
:103717008C598D5AE55A455960137406C3955AFF5B
:10372700E49559FE8E598F5A785B126AECE572A8B8
:103737005BB80015D3955C4010E572C3955CFFE458
:10374700955BFE8E5B8F5C8010E572243CC3955CB5
:10375700FFE4955BFE8E5B8F5CAE5BAF5C743B6F8B
:103767004E6006743C6F4E701AAE5BAF5C743B6F75
:103777004E70057572018003757202755C3A755B50
:10378700008003757200229000A0E0B40104C2100B
:103797008002D2109000A1E0B40104C2118002D2CD
:1037A700119000DEE075F0DCA4FFAEF0740A8E0421
:1037B7008F05FF126A889007C6ECF0A3EDF0A20D03
:1037C700401674038C068D07126A9874011200392B
:1037D7009007C4EEF0A3EFF07E017F0090009CE01D
:1037E700126A989000DFE08E048F05FF126A8874D2
:1037F7000AFF126A888D5F9000E8E075F0DCA4FF8D
:10380700AEF0740A8E048F05FF126A889007CAEC1F
:10381700F0A3EDF09000EAE060139000EAE0F5F025
:10382700741684FF7E00EF9007D4F08006746490CE
:1038370007D4F09000E0E0900084F090012AE09037
:10384700006EF09000B9E0900070F09000E2E09018
:103857000071F090008EE0900072F0900114E090FB
:103867000077F074E3900083F09000C9E0B40B0890
:1038770074E3900083F0805A9000C9E0B419129065
:1038870000DFE09068ED12008CE493900083F080F5
:10389700419000C9E0B41E129000DFE090690B125E
:1038A700008CE493900083F080289000C9E0B4284E
:1038B700129000DFE090693512008CE4939000834A
:1038C700F0800F9000C9E0B446089000C0E0900077
:1038D70083F0900087E0FE9000C6E0B506339000C5
:1038E70088E0FE9000F2E0B50627900089E0FE90A0
:1038F70000E4E0B5061B90008BE0FE900099E0B570
:10390700060F90008AE0FE9000D4E06E7003023A42
:10391700CB90005FE0C3940550087402900115F046
:10392700801C9000D4E0640360069000F2E0600819
:103937007406900115F08006740A900115F0900046
:10394700D4E0B403089000F2E064026002800674D9
:10395700009000F2F0900099E0B401067400900026
:10396700FFF0900099E0B4020674009000E4F09034
:103977000099E0B4030674009000F1F09000C6E0EF
:10398700601474199000ADF074009006DAF07400BA
:103997009006DBF0800C74009000ADF0741990066F
:1039A700DAF09000C6E0B40214741A9000AEF07416
:1039B700009006DEF074009006DFF0800C74009033
:1039C70000AEF0741A9006DEF09000E4E0D39401A4
:1039D7004014741B900117F074009006E2F0740015
:1039E7009006E3F0800C7400900117F0741B9006AA
:1039F700E2F09000F2E0B40114741C900118F07426
:103A0700009006E6F074009006E7F0800C740090D2
:103A17000118F0741C9006E6F09000D4E0B402069A
:103A27009000F2E06002801A74059006EAF07406CE
:103A37009006EEF074079006F2F074089006F6F020
:103A4700803074009006EAF074009006EBF0740082
:103A57009006EEF074009006EFF074009006F2F016
:103A670074009006F3F074009006F6F07400900668
:103A7700F7F0D22C9000C6E0900087F09000F2E0BB
:103A8700900088F09000E4E0900089F09000D4E086
:103A970090008AF0900099E090008BF0900099E0F8
:103AA70090006FF09000D4E0900073F09000F2E087
:103AB700900074F09000C6E0900075F09000E4E08C
:103AC700900076F09000FCE0B40117900027740F87
:103AD700F0A374FFF0900029E4F0A3F074029000C3
:103AE700FCF09000FCE0B40341900029E0FEA3E065
:103AF700FF900027E0FCA3E0FD126AE47410126A4D
:103B0700987408120039EF900080F0EF700674FF88
:103B1700900080F074009000FCF0900028E0900086
:103B270081F0900027E0900082F090008DE09000F7
:103B37004BF090004BE0240F90004CF090004BE0CE
:103B4700241E90004DF090004BE0242D90004EF085
:103B570090004CE0D3943C400B90004CE0C3943C65
:103B670090004CF090004DE0D3943C400B90004DFA
:103B7700E0C3943C90004DF090004EE0D3943C405D
:103B87000B90004EE0C3943C90004EF0900053E43D
:103B9700F090004BE0643B600790004BE0B43C20A2
:103BA70090004BE0B43B067402900053F090004B3A
:103BB700E0B43C069000537401F090004B7401F0A0
:103BC700900054E4F090004CE0643B600790004C98
:103BD700E0B43C2090004CE0B43B067402900054E3
:103BE700F090004CE0B43C069000547401F0900053
:103BF7004C7401F0900055E4F090004DE0643B6098
:103C07000790004DE0B43C2090004DE0B43B0674B3
:103C170002900055F090004DE0B43C0690005574BA
:103C270001F090004D7401F090004EE0643B600796
:103C370090004EE0B43C2090004EE0B43B06740286
:103C4700900056F090004EE0B43C06900056740188
:103C5700F090004E7401F090008DE0FE9000F0E0CF
:103C67002E900058F0900058E0641E6007900058AE
:103C7700E0B43C06900058E004F0900058E0641D62
:103C87006007900058E0B43B06900058E014F090AD
:103C97000058E0D3943C400B900058E0C3943C900C
:103CA7000058F0900058E0D3941E400D900058E063
:103CB700C3941E900059F0800A900058E0241E908B
:103CC7000059F075501E9000D3E090004FF090001F
:103CD7004FE075F00F84AFF07E00EF4E7006900056
:103CE7004FE004F090004FE00475F00F84AFF07ED2
:103CF70000EF4E700690004FE014F090004FE0B4D4
:103D0700790690004F7401F090004FE0D3943C4047
:103D17000F90004FE0C3943C90004FF0D2268002F2
:103D2700C22690004FE0240F900050F090004FE023
:103D3700241E900051F090004FE0242D900052F087
:103D4700900050E0D3943C400B900050E0C3943C6B
:103D5700900050F0900051E0D3943C400B900051FC
:103D6700E0C3943C900051F0900052E0D3943C4063
:103D77000B900052E0C3943C900052F022C293C2D1
:103D870094C291C292C287C290E5B554EFF5B5E5EA
:103D9700B554DFF5B5C296C295C2A0C297C2A2C2FA
:103DA700A1E5B554BFF5B5E5B5547FF5B5E5B5540F
:103DB700FBF5B5C212755D469000D6E07005756CCF
:103DC700028003756C0375540075530090001074DE
:103DD700FFF0A374DCF0C219C21BC21DC21F74C856
:103DE70090003BF074C890003FF074C8900043F017
:103DF70074C8900047F0755200755100C20D7546A2
:103E070000E56EB40903756E0075620090001DE44D
:103E1700F0A3F0756F10C215C216C217C21890072B
:103E2700C6E0FEA3E0FF7403126A9874011200391A
:103E37009007C4EEF0A3EFF0C20275560075550067
:103E4700900014E4F0A3F0C22D7558007557009048
:103E57000098E075F032A4FDACF0900025ECF0A3DB
:103E6700EDF0C23D2285F97285FA737E017F00E588
:103E770073126A98E5722FFF50010E8E598F5AAC54
:103E87005BAD5CEF2DFDEE3CFC8C5B8D5C123697D9
:103E97001236A21236AD1236B89000D4E0B4032C15
:103EA70075A71085F97285FA737E017F00E5731295
:103EB7006A98E5722FFF50010E8E598F5A1236C33A
:103EC7001236CE1236D91236E875A7002275A7101A
:103ED70085F97285FA737E017F00E573126A98E5AA
:103EE700722FFF50010E8E598F5A7E017F769001F7
:103EF70011E0126A98AC59AD5AED2FFFEC3EFE8ED9
:103F07005B8F5CE55CF5FDE55BF5FE900084E4F016
:103F170075A700741290005BF02285F97285FA7319
:103F27007E017F00E573126A98E5722FFF50010E3C
:103F37008E598F5A9007C6E0FCA3E0FDEF2DFDEEEA
:103F47003CFC8C5B8D5CE55CF5FDE55BF5FE2205D5
:103F570063229000D4E0640360079000F2E0B402AB
:103F67001EA2D8B34002C293A2D9B34002C294A200
:103F7700DAB34002C291A2DBB34002C2928044A2EC
:103F8700D8B3400AC2939000F2E06002C287A2D978
:103F9700B3400AC2949000F2E06002C290A2DAB382
:103FA700400EC2919000F2E06006E5B554EFF5B51A
:103FB700A2DBB3400EC2929000F2E06006E5B55472
:103FC700DFF5B5A2DCB34008C296C295C2A0C2977E
:103FD70075D8402285A77175A7109000D4E06403B7
:103FE70060079000F2E0B40224A2D8B34002C2876F
:103FF700A2D9B34002C290A2DAB34006E5B554EFA6
:10400700F5B5A2DBB34006E5B554DFF5B5A2DCB3E1
:1040170040089000E0E0900084F075D8408571A7D3
:1040270022900047E4936406600280FE74C89007FC
:10403700CCF8E4F0E8A3F075B50075840175A70026
:1040470075FFA0900057E4F075C91075A70F75A10B
:10405700C775A70075D90075CE0C75A70F75F1FE4A
:1040670075F2FF75F30775F47875A4BA75A5FF7532
:10407700A60775AE0075AFFF75D48175D5FF75D6E8
:10408700FF75D7FF75A70075A20175A14775F809D8
:1040970075D80075D90475DA0975DB0975DC0975FA
:1040A700DD0975DE0975D84075A71075D80075D973
:1040B7000475DA0975DB0975DC0975DD0975DE0933
:1040C70075D84075A70075E60875E71075BC0175CA
:1040D700BE0475BD6C75BE0775BDA075BE0875BD00
:1040E7000175BC0075BB1875BC2075BA0875E880EA
:1040F70075D11375A70F75E10575E20075C74012F5
:104107003D84759700759780740A126A787597C011
:10411700E5975420700280F8758F0275A700D2AF1B
:1041270075980075A90C75A70F75AB4375ADFB7531
:10413700AC1E75A71075C91875CA0075CB0075C870
:104147000475A700758912758E04758C00758A0031
:10415700C2A9D28C758D00758B00D2ABD28E75EF4C
:104167000675D944C29974C8F5097508001200E3A9
:1041770075B5001204E374639007CCF8E4F0E8A384
:10418700F012036F74C89007CCF8E4F0E8A3F0745A
:1041970064F5097508001200E390006FE09000993C
:1041A700F0C223900099E0D3940340067400900076
:1041B70099F0900099E09062EAF82828738028A285
:1041C700B44002D223802075A70F75F30F75A7009F
:1041D700A2A34002D223800F75A70F75F31775A707
:0741E70000A2A44002D22354
:0C62EA000241C40241C60241CE0241DF65
:1041EE00A223B34066757208E572D3940E5020E593
:1041FE00729007CCF8E4F0E8A3F012023E7464F576
:10420E00097508001200E37872740126F650D9740D
:10421E00029000D5F0900099E0D39403400674000C
:10422E00900099F0900099E09062F6F8282873803B
:10423E001674009000FFF0800E74009000E4F08081
:07424E000674009000F1F07E
:0C62F60002423D02423F02424702424F7A
:10425500D2228064757201E572D394075020E5720D
:104265009007CCF8E4F0E8A3F012023E7464F50977
:104275007508001200E37872740126F650D97401AE
:104285009000D5F0900099E0D39403400674009017
:104295000099F0900099E0906302F8282873801641
:1042A50074009000FFF0800E74009000E4F080062A
:0642B50074009000F1F01E
:0C6302000242A30242A50242AD0242B5D5
:1042BB00C22290006EE090012AF090006FE0900017
:1042CB0099F0900070E09000B9F0900071E09000D0
:1042DB00E2F0900072E090008EF0900073E090009E
:1042EB00D4F0900074E09000F2F0900075E0900034
:1042FB00C6F0900076E09000E4F0900077E090013B
:10430B0014F09000DFE07006740A9000DFF090006C
:10431B00C0E0700674E39000C0F09000C6E004901B
:10432B000087F012378EE5B54401F5B574069000A1
:10433B005DF0740190005EF07403900060F0740502
:10434B00900061F0741F900062F07405900063F0B0
:10435B0090005FE0B404067404900063F074009066
:10436B000064F07400900069F0740090006AF074BF
:10437B000190006BF0740090006CF074FF90006D76
:10438B00F07436900163F07430900164F0742D90EA
:10439B000165F07432900166F07420900167F0743F
:1043AB0038900168F07443900169F0747990016A58
:1043BB00F0746C90016BF0742090016CF074209091
:1043CB00016DF0742090016EF0742090016FF07409
:1043DB0020900170F07420900171F09000FBE09040
:1043EB000080F09000B2E0900081F09000B3E0907C
:1043FB000082F0A2B6B3920EA2B3B3920FA2A4B3F3
:10440B009229A2B4B3922AA2A3B3922B90007CE47C
:10441B00F0756E00743A90078CF074FD90078DF078
:10442B0090007DE4F09007C6E0FEA3E0FF7403125A
:10443B006A9874011200399007C4EEF0A3EFF0757F
:10444B006D0190005BE4F0C228756200C213D214B8
:10445B00C202757000C22FD203C230D204C231D255
:10446B0005C232D206C233D207C234D208C235D209
:10447B0009C236D20AC237D20BC238D20CC224C2FE
:10448B0025C226C227C22C12009E755E00756A00DB
:10449B00756000756432756500756600756700752B
:1044AB00680075690090001DE4F0A3F0756B00D2F5
:1044BB00B2D2A4D2B0D2B1D2A3D2A7D2A6D2A5D215
:1044CB00B7900098E0D394FA400674FA900098F0F5
:1044DB007E017F00900082E0126A98900081E02FAD
:1044EB00FF50010E900027EEF0A3EFF0EFD394FFF7
:1044FB00EE940F4007900027E4F0A3F0900080E0CB
:10450B00700674FF900080F074009000BFF0900074
:10451B00D5E0D39402400674019000D5F09000D6FC
:10452B00E07005756C028003756C039000D7E0D3C7
:10453B009401400674009000D7F09000DDE0C39426
:10454B000A5006740A9000DDF09000E7E0700674E4
:10455B00019000E7F09000E7E0B4FF0674FE9000D6
:10456B00E7F09000EEE0D394FE400674FE9000EE70
:10457B00F0900114E0D3940240067401900114F002
:10458B0090012AE0D394014006740190012AF07443
:10459B00019000F4F074019000F5F074009000FCB1
:1045AB00F0740090011CF074299006D2F0742A90DC
:1045BB0006D6F0D29C9000C7E0D394044006740456
:1045CB009000C7F09000F9E0D39404400674049077
:1045DB0000F9F0E56FD394104003756F109006D37C
:1045EB00E0D3940C400674009006D3F09006D7E00D
:1045FB00D3940C400674009006D7F09006DBE0D302
:10460B00940C400674009006DBF09006DFE0D39428
:10461B000C400674009006DFF09006E3E0D3940C98
:10462B00400674009006E3F09006E7E0D3940C404C
:10463B000674009006E7F09006EBE0D3940C40066E
:10464B0074009006EBF09006EFE0D3940C400674E8
:10465B00009006EFF09006F3E0D3940C4006740044
:10466B009006F3F09006F7E0D3940C40067400909C
:10467B0006F7F0D2EC75CF01A298B34005C29812A1
:10468B000616E54D6006A299B3B340028005C299A8
:10469B00120AB4E54E64016005E54EB4040280D500
:1046AB00C28E7E107F00E563126A98E58D75F0105F
:1046BB00A4FDACF0EF2DFDEE3CFCE58B75F010840A
:1046CB00FF7E00ED2FFFEC3EFE8E538F54D28E906B
:1046DB0000B9E060099000B9E0C3943D4002805CF2
:1046EB0090001F126AA690001FE0FEA3E0FF90004F
:1046FB0021E0FCA3E0FDEFB50542EEB5043EB2218F
:10470B00A20DB3401975E700A221B34008E5B544EB
:10471B0004F5B58006E5B554FBF5B575E7109000CB
:10472B0021E0FEA3E0FF900023E0FCA3E0FDEF2DD2
:10473B00FDEE3CFC900021ECF0A3EDF09000C6E008
:10474B0060099000C6E0C394034002806F1229C039
:10475B00A20DB3500990007CE0C3942B400280065D
:10476B009000B0E0F545E54575F005A4FFAEF0907F
:10477B0007CEEEF0A3EFF090009DE0C395604007ED
:10478B00E55EC3955F50079007CEE4F0A3F0AE2E25
:10479B00AF2F9007CEE0FCA3E0FDEFD39DEE9C4046
:1047AB0004C2A1800B90007CE0C394415002D2A1C3
:1047BB009000C6E0B40205A2A1B392A29000C6E09D
:1047CB00B4031C122ADBAE2EAF2F9007CEE0FCA356
:1047DB00E0FDEFD39DEE9C4004D2A18002C2A190DC
:1047EB0000A1E06009A2B3300F01B3B340028039DE
:1047FB00A2B3300F01B34031A2B3301101B3401C4F
:10480B009000D4E0B40306A224B3B3400280067434
:10481B000490005BF0D224A211B3920FA211B3301B
:10482B00B301B34004A211920FA2B6300E01B350E4
:10483B0003024EFEA2B6300E01B35003024EFEA28F
:10484B00B6301001B35003024D06756D009000B9E0
:10485B00E0B43D1975E700A210B34008E5B554FB71
:10486B00F5B58006E5B54404F5B575E710055DA211
:10487B0012B3B35013AE53AF54900010E0FCA3E04F
:10488B00FDEDC39FEC9E40030249E3E56CB4032EA0
:10489B00A22DB34022E55DB43B03756C01E55DC30E
:1048AB00943B500690005B7401F0E55DD3943B4064
:1048BB0006740290005BF0755D01D22D805EE56C95
:1048CB00B40206756C01755D3BE55DB43B05755D2A
:1048DB0001804990005BE07034E55DC3943B50066A
:1048EB0090005B7401F0E55DD3943B40067402903D
:1048FB00005BF0E55DC3943B5002D228E55DD39499
:10490B003B4002D228C296C295C2A0C2979000D655
:10491B00E0B40105123D848003755D01AE55AF56C1
:10492B00AC53AD54EF2DFDEE3CFC74028C068D07A1
:10493B001200398E558F569000B9E060099000B97E
:10494B00E0C3943D4002804390001FE0FEA3E0FFD4
:10495B009000B9E08E048F05FF126A8874018C06F3
:10496B008D07120039900023EEF0A3EFF090002397
:10497B00E0F8A3E0900021C8F0A3C8F090001FE47A
:10498B00F0A3F0C221E5B554FBF5B5A2B4B34002D8
:10499B00C22AA2A4B34002C229A2A3B34002C22BD3
:1049AB00A228B34002C228A224B34006A226922515
:1049BB008002B2259000A1E06012E56C700EA2247B
:1049CB00B35009A225302601B3B34002800674050B
:1049DB0090005BF0C224803AAE55AF56AC53AD5449
:1049EB00EF2DFDEE3CFC74018C068D071200398E09
:1049FB00558F56E56CC39402500DAC53AD5474B83F
:104A0B00C39D740B9C40028009123D847406900078
:104A1B005BF0E55DB43B12740390005BF0D2289021
:104A2B0000D6E0B40103123D84AE57AF58AC53AD82
:104A3B0054EF2DFDEE3CFC8C578D58AE53AF54EF1D
:104A4B00D39DEE9C4011900017E0FAA3E0FBEBC363
:104A5B0094E8EA940340028006900017126AA6902D
:104A6B000014E0FEA3E0FFAC53AD54EF2DFDEE3C84
:104A7B00FC900014ECF0A3EDF09000D6E0B401181C
:104A8B00AE53AF547405126A98740112003990003A
:104A9B0010EEF0A3EFF08011AE53AF547402126A14
:104AAB0098900010EEF0A3EFF0C28E758D00758B11
:104ABB0000756300755401755300D28EE55D240EAD
:104ACB0075F00F84AFF07E00EF4E7075900014E020
:104ADB00F8A3E0900012C8F0A3C8F0900012E0FE1B
:104AEB00A3E0FFEF4E600B7C7A7DF81269868E5146
:104AFB008F52900014E4F0A3F0AE51AF527428BE65
:104B0B0000039F5010E5622FFF50010E740112003D
:104B1B00398E518F528552629000DDE0A851B8005A
:104B2B000DD395524008E55290005AF08009900041
:104B3B00DDE01490005AF0E56C600675520075517B
:104B4B00009000D4E0B4030890004FE0655D600274
:104B5B00800BA225B34004D2278002B227E55D6407
:104B6B000B6005E55DB429099000C6E060031220D7
:104B7B002B900058E0655D6007900059E0B55D0330
:104B8B00756E00A213B35006A212B3B34003024CCE
:104B9B0041900092E0B40173900114E0B40214123E
:104BAB000C55900085E075F0BEA4FFAEF08E5B8FC8
:104BBB005C8056E56675F00A84FF7E0090058C12CA
:104BCB006ABFE0F55A755900AE59AF5A9000B7E07D
:104BDB00126A9874648E048F05FF126A888C5B8D41
:104BEB005CE55C900016F0AE59AF5A900090E01265
:104BFB006A9874648E048F05FF126A8874BE8C06E3
:104C0B008D07126A988E5B8F5C8017900090E07511
:104C1B00F0BEA4FFAEF08E5B8F5C9000B7E090000F
:104C2B0016F0E560C394CC5006900090E0700280C3
:104C3B0003123E6CD213E56CB40106E55D641160A2
:104C4B00028009756F0190005C7401F0E56C6003E4
:104C5B00024D019000D9E0600D900084E0A851B89E
:104C6B0000069552400280489000D9E0B40227908C
:104C7B00004BE0655D601790004CE0655D600F9048
:104C8B00004DE0655D600790004EE0B55D03756F0C
:104C9B0003756B00800CC200756B0090001DE4F077
:104CAB00A3F0900084E06006740990005BF08046EE
:104CBB0090004BE0B55D0B756F0190005C7401F0DB
:104CCB00803490004CE0B55D0B756F017402900061
:104CDB005CF0802290004DE0B55D0B756F017403A5
:104CEB0090005CF0801090004EE0B55D09756F018F
:104CFB00740490005CF0A210B3920EA210B330B605
:104D0B0001B35003024EFE756D019000B9E0B43D46
:104D1B001975E700A210B34008E5B54404F5B5805A
:104D2B0006E5B554FBF5B575E710E5B54401F5B5EA
:104D3B00742B90007CF0A210920EE55DD3944A4048
:104D4B0014D212E55DD39485400B740490005BF094
:104D5B00D228755D469000E1E0B40107E569C39484
:104D6B001440028009123D84741390005BF0A22F53
:104D7B00300301B3501D75E700A22FB34008E5B512
:104D8B004408F5B58006E5B554F7F5B575E710A2FF
:104D9B002F9203A230300401B3501D75E700A230EF
:104DAB00B34008E5B54402F5B58006E5B554FDF50D
:104DBB00B575E710A2309204A231300501B3500F44
:104DCB00A231B34004D2A28002C2A2A2319205A2A8
:104DDB0032300601B3500FA232B34004D2A180028D
:104DEB00C2A1A2329206A233300701B3501D75E760
:104DFB0000A233B34008E5B54440F5B58006E5B5F0
:104E0B0054BFF5B575E710A2339207A234300801F1
:104E1B00B3501D75E700A234B34008E5B54480F5E7
:104E2B00B58006E5B5547FF5B575E710A234920849
:104E3B00A235300901B3500FA235B34004D287809D
:104E4B0002C287A2359209A236300A01B3500FA2D3
:104E5B0036B34004D2908002C290A236920AA23797
:104E6B00300B01B3501D75E700A237B34008E5B511
:104E7B004410F5B58006E5B554EFF5B5A237920BA6
:104E8B0075E710A238300C01B3501D75E700A2383E
:104E9B00B34008E5B54420F5B58006E5B554DFF51C
:104EAB00B5A238920C75E710E569C39441500974AB
:104EBB000E90005BF0123D84900063E0FE90005F6B
:104ECB00E004C39E400990005FE0D3940640097450
:104EDB00FB90005BF0123D84900068E06015900041
:104EEB0068E0FE900062E06E600974FE90005BF07B
:104EFB00123D84A228B34008C296C295C2A0C297A5
:104F0B00900111E0600CAE51AF527414BE00059FBE
:104F1B0040028048900099E090630EF82828738037
:104F2B003BA2B4B35005A22AB340028005123ED473
:104F3B00D22A8028A2A3B35005A22BB3400280052E
:104F4B00123ED4D22B8015A2A4B35005A229B34094
:0C4F5B00028005123ED4D22980028000A2
:10630E00024F2A024F2C024F3F024F52024F65029C
:02631E004F67C7
:104F6700A215B3B3500890004FE0655D600302508F
:104F77003CA201B35006A200B3B3400302503490E1
:104F870000D4E0B4036EA20DB34038A227B34008A3
:104F970012363A12369780091236671236C375A74A
:104FA700009000F2E0B4011975E700A202B34008CF
:104FB700E5B54480F5B58006E5B5547FF5B575E7E9
:104FC70010802F12363A1236971236671236C3758B
:104FD700A7009000F2E0B4011975E700A202B34000
:104FE70008E5B54480F5B58006E5B5547FF5B57598
:104FF700E71080399000F2E0C39402500F12363A5E
:10500700123697A202B34002D287802112363A1293
:105017003697123667AE59AF5AAC2CAD2DEF2DFD32
:10502700EE3CFC8C5B8D5C1236C375A700C215D2B3
:1050370016D217D218A216B3B35008900050E065E5
:105047005D6003025111A201B35006A200B3B34041
:10505700030251099000D4E0B4036EA20DB34038A7
:10506700A227B3400812363A1236A28009123667D1
:105077001236CE75A7009000F2E0B4011975E7006B
:10508700A202B34008E5B54480F5B58006E5B554FE
:105097007FF5B575E710802F12363A1236A2123611
:1050A700671236CE75A7009000F2E0B4011975E7D4
:1050B70000A202B34008E5B54480F5B58006E5B522
:1050C700547FF5B575E71080399000F2E0C394027C
:1050D700500F12363A1236A2A202B34002D2908083
:1050E7002112363A1236A2123667AE59AF5AAC2C95
:1050F700AD2DEF2DFDEE3CFC8C5B8D5C1236CE7535
:10510700A700D215C216D217D218A217B3B35008E8
:10511700900051E0655D60030251EAA201B35006B9
:10512700A200B3B340030251E29000D4E0B4036E8F
:10513700A20DB34038A227B3400812363A1236AD53
:1051470080091236671236D975A7009000F2E0B4CD
:10515700011975E700A202B34008E5B54480F5B52B
:105167008006E5B5547FF5B575E710802F12363AFE
:105177001236AD1236671236D975A7009000F2E0E5
:10518700B4011975E700A202B34008E5B54480F5FC
:10519700B58006E5B5547FF5B575E710803D9000FD
:1051A700F2E0C39402501312363A1236ADA202B39C
:1051B7004006E5B54410F5B5802112363A1236ADF2
:1051C700123667AE59AF5AAC2CAD2DEF2DFDEE3C24
:1051D700FC8C5B8D5C1236D975A700D215D216C22E
:1051E70017D218A218B3B35008900052E0655D605B
:1051F700030252C3A201B35006A200B3B340030295
:1052070052BB9000D4E0B4036EA20DB34038A2277E
:10521700B3400812363A1236B8800912366712368A
:10522700E875A7009000F2E0B4011975E700A20243
:10523700B34008E5B54480F5B58006E5B5547FF57C
:10524700B575E710802F12363A1236B81236671244
:1052570036E875A7009000F2E0B4011975E700A2DF
:1052670002B34008E5B54480F5B58006E5B5547F3F
:10527700F5B575E710803D9000F2E0C39402501336
:1052870012363A1236B8A202B34006E5B54420F505
:10529700B5802112363A1236B8123667AE59AF5A70
:1052A700AC2CAD2DEF2DFDEE3CFC8C5B8D5C1236EE
:1052B700E875A700D215D216D217C218E56F90630A
:0C52C70020F82828730258D89000F9E065
:066320000252CC0252CF34
:1052D300906353F8282873121B078012121B078050
:0E52E3000D121B918008121C3D8003121C3D11
:0F6353000252DA0252DF0252E40252E90252EE23
:1052F100756F020258D8121D69121E80A23DB3407B
:10530100229000BBE0F56B90008CE0256BFE9000D5
:105311005AE075F01E84FC7F00EE2CF53474109079
:10532100005BF09007C4E0FEA3E0FF740A126A98E4
:10533100900012E0FCA3E0FD74098F02FF126A885D
:105341008D078C038E048A058B061269869007C827
:10535100EEF0A3EFF09000E2E0B40108743CBE006F
:10536100059F4002800D743C9007C8F8E4F0E8A363
:10537100F0801B9007C8E0FEA3E0FF74F0BE0003BD
:105381009F500B74F09007C8F8E4F0E8A3F0E534FF
:1053910070037534019007C8E0FEA3E0FFE5342FE8
:1053A100FF50010E9007C8EEF0A3EFF0756F039068
:0353B100005CE0BD
:036326000252F729
:1053B400906362F82828738022A23E4003756F0A26
:1053C4008019A23E4003756F0B8010A23E40037506
:0B53D4006F0C8007A23E4003756F0DB8
:0F6362000253BB0253BD0253C60253CF0253D89E
:1053DF000258D89006D3E06003122114900112E016
:1053EF00B40114900113E0A851B80004955250076E
:1053FF00E55EC3955F4002800302548C9000C7E0C6
:10540F00D39402403F90009BE02403A851B80004BE
:10541F009552500990009DE0D3956050028008D2BC
:10542F0001740890005BF090009BE0A851B8000554
:10543F00D39552500B90009DE02403C3956050020A
:10544F00C201803990009BE02403A851B800049555
:10545F00525007E55EC3955F40028008D201740881
:10546F0090005BF090009BE0A851B80005D39552D7
:10547F005009E55F240FC3955E5002C2019000E111
:10548F00E07007E569C3941440028002D201A201C3
:10549F004005756F04800A756F1090001DE4F0A32E
:1054AF00F0A20DB34029E56675F00A84FF7E0090E7
:1054BF00058C126ABFE0C394695005122060800FFB
:1054CF009007C6E0F8A3E09007C4C8F0A3C8F002A5
:0654DF0058D89000C7E060
:066329000253E20254E100
:1054E500906371F8282873120D3F8012120D3F80CA
:0E54F5000D120EED8008120F9F8003120F9F04
:0F6371000254EC0254F10254F60254FB025500A0
:105503009006D7E060031221F0756F050258D81298
:1055130010AB756F069006DBE060031222E0900685
:10552300DFE060031223BC0258D8900016E0600647
:10553300A20DB3B34002801D900016E02529FFAEF3
:105543002850010E8E288F29E55DD3940F500690C5
:105553000016E014F01212F1756F079006E3E06095
:10556300031224989006E7E060031225740258D8CA
:10557300900114E0B40203120CCD12154E756F089E
:105583009006EBE060031226509006EFE0600312F2
:10559300272C0258D812190AA215B35005A216B324
:1055A30040028008D215D216D217D218756F109008
:1055B30006F3E060031228089006F7E06003122860
:1055C300E40258D80258D890003DE0C394465008EE
:1055D300C296744690003DF0900053E0B4011DE57F
:1055E300342406F5349007C8E0FEA3E0FF74062FC9
:1055F300FF50010E9007C8EEF0A3EFF0900053E0C8
:10560300B4021DE534240CF5349007C8E0FEA3E092
:10561300FF740C2FFF50010E9007C8EEF0A3EFF0BC
:1056230085345A75590090004BE0F5721236F7E550
:105633005C90003DF0900008E559F0A3E55AF0E5D1
:105643007290003EF0C21A9007C8E0F559A3E0F546
:105653005A90004BE0F5721236F7E55C90003BF090
:10566300900000E559F0A3E55AF0E57290003CF094
:10567300C219E56CB40105756F0B8003756F0302E6
:1056830058D8900041E0C3944650139000E2E0B430
:105693000104C2968002C2957446900041F09000C6
:1056A30054E0B4011DE5342406F5349007C8E0FE48
:1056B300A3E0FF74062FFF50010E9007C8EEF0A37E
:1056C300EFF0900054E0B4021DE534240CF534905F
:1056D30007C8E0FEA3E0FF740C2FFF50010E9007F4
:1056E300C8EEF0A3EFF085345A75590090004CE0F2
:1056F300F5721236F7E55C900041F090000AE55927
:10570300F0A3E55AF0E572900042F0C21C9007C87E
:10571300E0F559A3E0F55A90004CE0F5721236F724
:10572300E55C90003FF0900002E559F0A3E55AF0E4
:10573300E572900040F0C21BE56CB40105756F0C77
:105743008003756F030258D8900045E0C394465018
:10575300139000E2E0B40104C2968002C2A0744632
:10576300900045F0900055E0B4011DE5342406F5A2
:10577300349007C8E0FEA3E0FF74062FFF50010E2C
:105783009007C8EEF0A3EFF0900055E0B4021DE5DA
:1057930034240CF5349007C8E0FEA3E0FF740C2F0B
:1057A300FF50010E9007C8EEF0A3EFF085345A7551
:1057B300590090004DE0F5721236F7E55C90004514
:1057C300F090000CE559F0A3E55AF0E5729000461D
:1057D300F0C21E9007C8E0F559A3E0F55A90004DBA
:1057E300E0F5721236F7E55C900043F0900004E5B3
:1057F30059F0A3E55AF0E572900044F0C21DE56C40
:10580300B40105756F0D8003756F030258D89000BE
:1058130049E0C3944650139000E2E0B40104C296F9
:105823008002C2977446900049F0900056E0B4019C
:105833001DE5342406F5349007C8E0FEA3E0FF74A9
:10584300062FFF50010E9007C8EEF0A3EFF0900073
:1058530056E0B4021DE534240CF5349007C8E0FE8D
:10586300A3E0FF740C2FFF50010E9007C8EEF0A3C6
:10587300EFF085345A75590090004EE0F5721236F8
:10588300F7E55C900049F090000EE559F0A3E55A66
:10589300F0E57290004AF0C2209007C8E0F559A3E2
:1058A300E0F55A90004EE0F5721236F7E55C900091
:1058B30047F0900006E559F0A3E55AF0E572900031
:1058C30048F0C21FE56CB40103756C00756F03806B
:0558D3000480028000CA
:10632F0002551202552D0255730255980255C70298
:10633F0055CA02568502574B0258110258D40258BB
:04634F00D60258D842
:1058D80090003BE0B55D02800302597AA21940723C
:1058E800900000E0FEA3E0FFEF4E6021AE55AF56FA
:1058F800900000E0FCA3E0FD12000374068E048F04
:1059080005FF126A88900000ECF0A3EDF090003CCF
:10591800E0601A900000E0FEA3E0FFAC55AD56EF42
:105928002DFDEE3CFC900000ECF0A3EDF090003C67
:10593800E0D39401401A900000E0FEA3E0FFAC55CC
:10594800AD56EF2DFDEE3CFC900000ECF0A3EDF021
:10595800D219AE53AF54900000E0FCA3E0FDEFC3B2
:105968009DEE9C400D123F21D296C21974C890003A
:105978003BF0A219B3B3500790003BE0B55D02803D
:105988000D123F21D29674C890003BF0C2199000C6
:105998003DE0B55D028003025A35A21A40729000BC
:1059A80008E0FEA3E0FFEF4E6021AE55AF56900031
:1059B80008E0FCA3E0FD12000374068E048F05FFC7
:1059C800126A88900008ECF0A3EDF090003EE060C9
:1059D8001A900008E0FEA3E0FFAC55AD56EF2DFD90
:1059E800EE3CFC900008ECF0A3EDF090003EE0D314
:1059F8009401401A900008E0FEA3E0FFAC55AD56B4
:105A0800EF2DFDEE3CFC900008ECF0A3EDF0D21A6F
:105A1800AE53AF54900008E0FCA3E0FDEFC39DEE49
:105A28009C400AC296744690003DF0C21AA21AB36E
:105A3800B3500790003DE0B55D02800AC2967446F7
:105A480090003DF0C21A90003FE0B55D028003026D
:105A58005AFBA21B4072900002E0FEA3E0FFEF4E4B
:105A68006021AE55AF56900002E0FCA3E0FD1200A5
:105A78000374068E048F05FF126A88900002ECF00A
:105A8800A3EDF0900040E0601A900002E0FEA3E071
:105A9800FFAC55AD56EF2DFDEE3CFC900002ECF04E
:105AA800A3EDF0900040E0D39401401A900002E08A
:105AB800FEA3E0FFAC55AD56EF2DFDEE3CFC90008B
:105AC80002ECF0A3EDF0D21BAE53AF54900002E00D
:105AD800FCA3E0FDEFC39DEE9C4018123F2190000F
:105AE800E2E0B40104D2968002D295C21B74C89039
:105AF800003FF0A21BB3B3500790003FE0B55D0232
:105B08008018123F219000E2E0B40104D29680028E
:105B1800D29574C890003FF0C21B900041E0B55D7B
:105B2800028003025BCCA21C407290000AE0FEA334
:105B3800E0FFEF4E6021AE55AF5690000AE0FCA39F
:105B4800E0FD12000374068E048F05FF126A889028
:105B5800000AECF0A3EDF0900042E0601A90000A11
:105B6800E0FEA3E0FFAC55AD56EF2DFDEE3CFC90FA
:105B7800000AECF0A3EDF0900042E0D39401401A43
:105B880090000AE0FEA3E0FFAC55AD56EF2DFDEE08
:105B98003CFC90000AECF0A3EDF0D21CAE53AF54DD
:105BA80090000AE0FCA3E0FDEFC39DEE9C40159039
:105BB80000E2E0B40104C2968002C29574469000E7
:105BC80041F0C21CA21CB3B35007900041E0B55D80
:105BD8000280159000E2E0B40104C2968002C295EA
:105BE8007446900041F0C21C900043E0B55D02800D
:105BF80003025C9DA21D4072900004E0FEA3E0FF3A
:105C0800EF4E6021AE55AF56900004E0FCA3E0FDD6
:105C180012000374068E048F05FF126A8890000430
:105C2800ECF0A3EDF0900044E0601A900004E0FE70
:105C3800A3E0FFAC55AD56EF2DFDEE3CFC90000403
:105C4800ECF0A3EDF0900044E0D39401401A9000EA
:105C580004E0FEA3E0FFAC55AD56EF2DFDEE3CFC95
:105C6800900004ECF0A3EDF0D21DAE53AF549000B9
:105C780004E0FCA3E0FDEFC39DEE9C4018123F2119
:105C88009000E2E0B40104D2968002D2A0C21D7452
:105C9800C8900043F0A21DB3B35007900043E0B58D
:105CA8005D028018123F219000E2E0B40104D29610
:105CB8008002D2A074C8900043F0C21D900045E055
:105CC800B55D028003025D6EA21E407290000CE07A
:105CD800FEA3E0FFEF4E6021AE55AF5690000CE0FA
:105CE800FCA3E0FD12000374068E048F05FF126A00
:105CF8008890000CECF0A3EDF0900046E0601A905C
:105D0800000CE0FEA3E0FFAC55AD56EF2DFDEE3CD8
:105D1800FC90000CECF0A3EDF0900046E0D3940169
:105D2800401A90000CE0FEA3E0FFAC55AD56EF2DF5
:105D3800FDEE3CFC90000CECF0A3EDF0D21EAE534F
:105D4800AF5490000CE0FCA3E0FDEFC39DEE9C4037
:105D5800159000E2E0B40104C2968002C2A0744625
:105D6800900045F0C21EA21EB3B35007900045E054
:105D7800B55D0280159000E2E0B40104C29680028D
:105D8800C2A07446900045F0C21E900047E0B55D81
:105D9800028003025E3FA21F4072900006E0FEA34D
:105DA800E0FFEF4E6021AE55AF56900006E0FCA331
:105DB800E0FD12000374068E048F05FF126A8890B6
:105DC8000006ECF0A3EDF0900048E0601A900006A1
:105DD800E0FEA3E0FFAC55AD56EF2DFDEE3CFC9088
:105DE8000006ECF0A3EDF0900048E0D39401401ACF
:105DF800900006E0FEA3E0FFAC55AD56EF2DFDEE9A
:105E08003CFC900006ECF0A3EDF0D21FAE53AF546B
:105E1800900006E0FCA3E0FDEFC39DEE9C40181245
:105E28003F219000E2E0B40104D2968002D297C2EA
:105E38001F74C8900047F0A21FB3B35007900047E3
:105E4800E0B55D028018123F219000E2E0B4010441
:105E5800D2968002D29774C8900047F0C21F900073
:105E680049E0B55D028003025F10A22040729000F5
:105E78000EE0FEA3E0FFEF4E6021AE55AF56900056
:105E88000EE0FCA3E0FD12000374068E048F05FFEC
:105E9800126A8890000EECF0A3EDF090004AE060E2
:105EA8001A90000EE0FEA3E0FFAC55AD56EF2DFDB5
:105EB800EE3CFC90000EECF0A3EDF090004AE0D32D
:105EC8009401401A90000EE0FEA3E0FFAC55AD56D9
:105ED800EF2DFDEE3CFC90000EECF0A3EDF0D2208F
:105EE800AE53AF5490000EE0FCA3E0FDEFC39DEE6F
:105EF8009C40159000E2E0B40104C2968002C2976B
:105F08007446900049F0C220A220B3B35007900015
:105F180049E0B55D0280159000E2E0B40104C29644
:105F28008002C2977446900049F0C2209000E4E0D5
:105F3800B40202800302606590007EE0D39565504C
:105F48006490007EE0F4042565FE9000E7E08E0092
:105F5800F5F0E884FF7E008F72EFC39410500CEFC9
:105F68008572F0A4FDACF08D7280037572FF90000D
:105F78007EE0D39572400B90007EE0C39572F57079
:105F88008003757000900102E0D39570400690017F
:105F980002E0F570900103E0C3957050069001038C
:105FA800E0F570807190007EE0C39565FE9000E793
:105FB800E08E00F5F0E884FF7E008F72EFC3941046
:105FC800500CEF8572F0A4FDACF08D7280037572F1
:105FD800FF85725A75590090007EE0255AFFAE5928
:105FE80050010E8E598F5A74FFBE0009D39F400589
:105FF800855A7080037570FF900102E0D395704058
:1060080006900102E0F570900103E0C39570500618
:10601800900103E0F570A20DB3B3500D90007FE03E
:10602800FE9000EFE0D39E5002800E740790005B54
:10603800F0E5B554BFF5B5802175A71075E700E503
:10604800CDC395704008E5B554BFF5B58006E5B5F4
:106058004440F5B575E71075A70075A700E56EC350
:106068009409500AA2EDB34005C2ED122C7AAE5342
:10607800AF547410C39F74279E400C90007DE0C3FA
:10608800945A40030262E7A212B34009123D847495
:106098000690005BF0A223B34008E5B54404F5B5CB
:1060A8008006E5B554FBF5B5A214B3500EE560D3F0
:1060B80094334007E560C394CC4002802FE5B54493
:1060C80001F5B5742B90007CF0900090E075F0BE5F
:1060D800A4FFAEF08E5B8F5C7402BE000AD39F40B3
:1060E80006755C02755B00123E6CD21490007DE070
:1060F800D394014007E560C3941A40028002C21499
:106108009006D3E06003122114A22F300301B3508C
:1061180017A22FB34008E5B54408F5B58006E5B5E4
:1061280054F7F5B5A22F92039006D7E06003122129
:10613800F0A230300401B35017A230B34008E5B5DF
:106148004402F5B58006E5B554FDF5B5A2309204D4
:106158009006DBE060031222E0A231300501B35063
:106168000FA231B34004D2A28002C2A2A23192058A
:106178009006DFE060031223BCA232300601B35060
:106188000FA232B34004D2A18002C2A1A232920669
:106198009006E3E06003122498A233300701B3505D
:1061A80017A233B34008E5B54440F5B58006E5B518
:1061B80054BFF5B5A23392079006E7E060031225B5
:1061C80074A234300801B35017A234B34008E5B5BF
:1061D8004480F5B58006E5B5547FF5B5A23492083C
:1061E8009006EBE06003122650A235300901B35047
:1061F8000FA235B34004D2878002C287A235920924
:106208009006EFE0600312272CA236300A01B35043
:106218000FA236B34004D2908002C290A236920AEE
:106228009006F3E06003122808A237300B01B35040
:1062380017A237B34008E5B54410F5B58006E5B5B3
:1062480054EFF5B5A237920B9006F7E060031228D9
:10625800E4A238300C01B35017A238B34008E5B5B2
:106268004420F5B58006E5B554DFF5B5A238920CA3
:1062780090007DE0C3945A5010E56EB4090990006F
:106288007DE004F0756E00803BE56EB40903756E21
:1062980000755400755300758D00758B007563008B
:1062A80090007CE0C39441500890007CE004F080AA
:1062B80006744190007CF090007CE0B44106E5B59E
:1062C80054FEF5B590007DE0D394014007E569C31D
:1062D800944140028009740E90005BF0123D8402E4
:0262E8004680EE
:106380000000010001400160018001A001C001E0A6
:1063900002000300039603B603D603F404000500CD
:1063A0000512052405360548055A056C057E05903D
:1063B00005A805C005DE0600061406280646066E7A
:1063C00006AE00FF013F015F017F019F01BF01DFBA
:1063D00001FF02FF039503B503D503F303FF04FF99
:1063E00005110523053505470559056B057D058F05
:1063F00005A705BF05DD05F1061306270645066D51
:1064000006AD06ED0FAA0FA50F9F0F9A0F940F8DE3
:106410000F870F800F780F710F680F600F570F4EA7
:106420000F450F3B0F300F250F1A0F0E0F020EF501
:106430000EE80EDB0ECC0EBE0EAE0E9F0E8E0E7D47
:106440000E6C0E5A0E470E340E200E0C0DF70DE298
:106450000DCB0DB50D9D0D850D6D0D540D3A0D2017
:106460000D050CE90CCE0CB10C940C760C580C3AC2
:106470000C1B0BFB0BDB0BBB0B9A0B790B570B3578
:106480000B130AF10ACE0AAB0A870A640A400A1CF7
:1064900009F809D409B0098C09670943091F08FBE9
:1064A00008D608B2088E086A0846082307FF07DCEA
:1064B00007B9079607730751072F070D06EC06CAA1
:1064C00006AA068906690649062A060A05EC05CDCC
:1064D00005B0059205750558053C0520050504EA3B
:1064E00004CF04B5049C04820469045104390422D5
:1064F000040B03F403DE03C803B2039D0389037591
:106500000361034D033B03280316030402F202E177
:1065100002D102C002B002A002910282027302659F
:1065200002570249023C022F02220216020901FD13
:1065300001F201E601DB01D001C601BB01B101A7F7
:10654000019D0194018B0182017901700168016054
:10655000015801500148014101390132012B012547
:10656000011E01180111010B010500FF00FA0FA621
:106570000FA00F990F920F8B0F840F7C0F740F6B6E
:106580000F620F580F4E0F430F380F2C0F1F0F12B3
:106590000F050EF70EE80ED80EC80EB70EA50E9317
:1065A0000E800E6C0E580E420E2C0E150DFD0DE4D5
:1065B0000DCB0DB10D950D790D5D0D3F0D200D012C
:1065C0000CE10CC00C9E0C7C0C590C350C100BEA29
:1065D0000BC40B9E0B760B4F0B260AFD0AD40AAA9E
:1065E0000A800A550A2A09FF09D409A8097C09501A
:1065F000092508F908CD08A10875084A081E07F3FF
:1066000007C8079D07730749072006F706CE06A6A9
:10661000067E06570630060A05E405BF059B05778A
:1066200005540532051004EF04CE04AE048F047146
:1066300004530435041903FD03E203C703AD0394B7
:10664000037B0363034B0334031E030802F302DEE0
:1066500002CA02B602A30291027F026D025C024CE2
:10666000023C022C021D020E020001F201E401D7DD
:1066700001CA01BE01B101A6019A018F0185017A0B
:1066800001700166015D0153014A01410139013187
:106690000129012101190112010B010400FD00F77C
:1066A00000F000EA00E400DE00D900D300CE00C90B
:1066B00000C400BF00BA00B500B100AD00A800A43E
:1066C00000A0009C009900950091008E008A008730
:0866D00000840081007E007BC4
:10009E007547009007D0E4F0A3F07531007530007D
:1000AE00754D00754E00C23AD23B74FE9007DAF8D9
:1000BE00E4F0E8A3F074FE9007DCF8E4F0E8A3F0B7
:1000CE00745A9007DEF0745A9007DFF0D23CC22EBD
:1000DE00C23EC23922750B00750A00AE0AAF0BACD8
:1000EE0008AD09EDC39FEC9E401674FF126A787539
:1000FE00CF01780B740126F6500418E436F650DB67
:10010E0022900057E0B4AA1C90078CE0B43C1590E6
:10011E0007CCE0FEA3E0FFEF4E6009741EBE0004A4
:10012E00D39F500302023D755C00755B0075F809A4
:10013E009007CCE0FEA3E0FF74076F4E6006740ECE
:10014E006F4E7006743A90078CF09007CCE0FEA3C9
:10015E00E0FF7408BE001ED39F401A7E017F0890F8
:10016E0007CCE0FCA3E0FD1DBDFF011C1200038EB9
:10017E00598F5A801F9007CCE0FEA3E0FF7408123F
:10018E006ADC8F048E057E017F08CDCCCD12000374
:10019E008E598F5AAE5BAF5C740CD39F74019E5018
:1001AE0003020238A2F9B3407EE55C455B7003752D
:1001BE00A382AE5BAF5C74016F4E700375A300AE8D
:1001CE005BAF5C74026F4E700D9007CDE075F00260
:1001DE00A4FDACF08DA3AE5BAF5C74036F4E7003E9
:1001EE0075A300AE5BAF5C7403BE00039F5013ACEF
:1001FE0059AD5AED2FFFEC3EFE900088126ABFE01B
:10020E00F5A3AE5BAF5CEFB40B09EEB4010574144D
:10021E00126A78AE5BAF5CEFB40B07EEB4010375F8
:10022E00F80D785B126AEC0201A2900057E4F022FE
:10023E00755C00755B0075F8099007CCE0FEA3E0D5
:10024E00FF7408BE001ED39F401A7E017F089007E0
:10025E00CCE0FCA3E0FD1DBDFF011C1200038E5976
:10026E008F5A801F9007CCE0FEA3E0FF7408126A3D
:10027E00DC8F048E057E017F08CDCCCD1200038E5F
:10028E00598F5AAE5BAF5C7411D39F74019E5003AD
:10029E0002036EA2F9B3500302036BE55C455B707B
:1002AE000375A3D2AE5BAF5C74016F4E700375A382
:1002BE0000AE5BAF5C74026F4E700D9007CDE075B3
:1002CE00F002A4FDACF08DA3AE5BAF5C74036F4E79
:1002DE00700375A300AE5BAF5C74046F4E70037554
:1002EE00A300AE5BAF5C74056F4E700375A300AEDA
:1002FE005BAF5C74066F4E700375A300AE5BAF5CB4
:10030E0074076F4E700375A300AE5BAF5C74086F1D
:10031E004E700375A300AE5BAF5C7408BE00039F06
:10032E005016AC59AD5AED2FFFEC3EFE90008312E5
:10033E006ABFE5A3F075A300AE5BAF5CEFB4100926
:10034E00EEB401057414126A78AE5BAF5CEFB410B4
:10035E0007EEB4010375F80D785B126AEC02029198
:10036E0022755C00755B0075F809AE5BAF5C7417A7
:10037E00BE0004D39F5003020447A2F9B3500302F8
:10038E000444E55C455B700375A3D2AE5BAF5C7451
:10039E00016F4E700375A300AE5BAF5C74026F4EBF
:1003AE00700D9007CDE075F002A4FDACF08DA3AEFC
:1003BE005BAF5C74036F4E700375A300AE5BAF5CF6
:1003CE0074046F4E700375A300AE5BAF5C74056F63
:1003DE004E700375A300AE5BAF5C74066F4E700378
:1003EE0075A300AE5BAF5C74076F4E700375A30010
:1003FE00AE5BAF5C74086F4E700375A300AE5BAF5F
:10040E005C7408BE00039F500C900065126ABFE535
:10041E00A3F075A300AE5BAF5C74166F4E700574DF
:10042E0014126A78AE5BAF5C74166F4E700375F87B
:10043E000D785B126AEC02037822900057E0B4ABA1
:10044E000280030204E2755C00755B0075F809AE6C
:10045E005BAF5C7412BE007CD39F4078A2F9B340B0
:10046E0070E55C455B700375A382AE5BAF5C740197
:10047E006F4E700375A300AE5BAF5C74026F4E706F
:10048E000D9007CDE075F002A4FDACF08DA3AE5B30
:10049E00AF5C74036F4E700375A300AE5BAF5C74FC
:1004AE0003BE00039F500990006A126ABFE0F5A3D5
:1004BE00AE5BAF5C74116F4E70057414126A78AE39
:1004CE005BAF5C74116F4E700375F80D785B126A3A
:1004DE00EC02045D229007D7E4F074649007CCF828
:1004EE00E4F0E8A3F012036F74C89007CCF8E4F0C0
:1004FE00E8A3F0900071E0B4371A90006EE090001F
:10050E0065F090006FE0900066F0900070E0900053
:10051E0067F080469007D77401F074659007CCF8A9
:10052E00E4F0E8A3F012036F74C89007CCF8E4F07F
:10053E00E8A3F0900071E0B4371A90006EE09000DE
:10054E0065F090006FE0900066F0900070E0900013
:10055E0067F0800674029007D7F09007D8E4F07425
:10056E00669007CCF8E4F0E8A3F012036F74C8901D
:10057E0007CCF8E4F0E8A3F0900070E0B4371290E6
:10058E00006EE090005FF090006FE0900068F080E9
:10059E00769007D87401F074679007CCF8E4F0E811
:1005AE00A3F012036F74C89007CCF8E4F0E8A3F040
:1005BE00900070E0B4371290006EE090005FF09003
:1005CE00006FE0900068F0803E74029007D8F074DF
:1005DE00689007CCF8E4F0E8A3F012036F74C890AB
:1005EE0007CCF8E4F0E8A3F0900070E0B437129076
:1005FE00006EE090005FF090006FE0900068F08079
:10060E000674039007D8F022E54E64046006E5995F
:10061E0064FF6002802AA23A4004D23A8020E54E5E
:10062E00600874E6254E90005BF0754E00E54D6057
:10063E000874F0254D90005BF0754D00C23A8002B3
:10064E00C23AE54E9033F8F8282873754E00E599B6
:10065E00B4FF03754D01E599B4FE03754D02E5999E
:10066E00B4FD03754D03E599B4FC03754D04E5998E
:10067E00B4FA03754D05E599B4FB06754E01123DAE
:10068E0084E599B4F906754E04123D84E599D39428
:10069E00E54007E599C394F04002801685994F75A1
:1006AE004E027E017F00E54FC394E6126A988E32A9
:1006BE008F339007D0E4F0A3F0E599D394C44007AC
:1006CE00E599C394E64002802885994F754E0374D0
:1006DE00E5C3954FF533753200AE32AF339063807C
:1006EE00126A67E493F87401939007D0C8F0A3C818
:1006FE00F0D299020AB390006EE070429007D0E0FB
:10070E00FEA3E0FF74FFBE00039F5009EFC39446A3
:10071E00EE940640119007D0E0FEA3E0FFEFD394D5
:10072E006DEE940640139007D0E0FEA3E0FF90001C
:10073E008C126ABFE599F08003859973801190073A
:10074E00D0E0FEA3E0FF90008C126ABFE599F09016
:10075E0007D0126AA69007D0E0FEA3E0FFEFB40127
:10076E0006EEB40702800302089B90078CE0B43CAF
:10077E00028003020885C29C90006EE090012AF070
:10078E0090006FE0900099F0900070E09000B9F04A
:10079E00900071E09000E2F0900072E090008EF018
:1007AE00900073E09000D4F0900074E09000F2F0AE
:1007BE00900075E09000C6F0900076E09000E4F0B6
:1007CE00900077E0900114F012378E900080E09048
:1007DE0000FBF0900081E09000B2F0900082E0907B
:1007EE0000B3F074639007CCF8E4F0E8A3F074ABB8
:1007FE00900057F0120448900057E4F075096475A4
:10080E0008001200E3A2224038757201E572D394FB
:10081E0007502CE5729007CCF8E4F0E8A3F074AA28
:10082E00900057F012010FE572C394075009750935
:10083E00647508001200E37872740126F650CD80BC
:10084E0036757208E572D3940E502CE5729007CC73
:10085E00F8E4F0E8A3F074AA900057F012010FE547
:10086E0072C3940E50097509647508001200E3787E
:10087E0072740126F650CD74C89007CCF8E4F0E8F7
:10088E00A3F0D29C754E00754D007599FB020AB30C
:10089E009007D0E0FEA3E0FFEF4E7006859931750C
:1008AE0030009007D0E0FEA3E0FF74016F4E701B86
:1008BE00AC30AD31AA32AB33ED2BFBEC3AFA8A06F3
:1008CE008B0790008C126ABFE599F09007D0126AE0
:1008DE00A69007D0E0FEA3E0FF74026F4E7021AC2D
:1008EE0030AD3174566D4C7006E54F64E660028093
:1008FE0003123D8412378E854F99754E00754D004B
:10090E00020AB39007D0E0FEA3E0FF90008C126ABB
:10091E00BFE599F09007D0126AA69007D0E0FEA32B
:10092E00E0FFAC32AD338F028E038C068D079063E1
:10093E00C2126A67E493F9740193FEEAD39EEB99AF
:10094E004009854F99754E00754D00020AB3900708
:10095E00D0E0FEA3E0FF90008C126ABFE599F09004
:10096E0007D0126AA69007D0E0FEA3E0FFEFB40016
:10097E0006EEB401028003020AB3900067E075F040
:10098E0002A4FDACF08D72ED90008C126ACAEDFAE5
:10099E00E0FBEA90008F126ACAEBFAE0FBEA2BFA50
:1009AE00900067E0B502028003020AA50DED9000EB
:1009BE008C126ACAE572FDE0FAED900090126ACAD6
:1009CE00EAFDE0FAEDC39AFD900067E0B5050280FE
:1009DE0003020AA5E57290008E126ACAE572FDE066
:1009EE00FAED900091126ACAEAFDE0FAED2AFD9046
:1009FE000067E0B505028003020AA5E57290009239
:100A0E00126ACAFDE0FAED900067E0F4042A900045
:100A1E006EF0E572900093126ACAFDE0FAED900056
:100A2E0067E0F4042A90006FF0E572900094126A69
:100A3E00CAFDE0FAED900067E0F4042A900070F031
:100A4E00E572900095126ACAFDE0FAED900067E03B
:100A5E00F4042A9007CCF8E4F0E8A3F074AB90000D
:100A6E0057F01204487509647508001200E39007E8
:100A7E00CC126AA61204487509647508001200E3C8
:100A8E009007CC126AA61204487599F97509647517
:100A9E0008001200E380FE7599FF75096475080061
:050AAE001200E380FED0
:0F33F80002065902070402089E02091102095C2D
:100AB30022E54D903407F8282873020B989007D04D
:100AC300E0FEA3E0FF90005D126ABFE0F599900796
:100AD300D0126AA69007D0E0FEA3E0FF74116F4E18
:100AE3007003754D00020B98856D99020B98900762
:100AF300D0E0FEA3E0FF90008C126ABFE0F599EF0F
:100B0300B40107EEB40703754D009007D0126AA62F
:070B1300020B989007D1E0EE
:0F340700020ABD020AC0020AEB020AF1020B160A
:100B1A009035BAF82828738552998067855E99803E
:100B2A0062856099805D856499805885669980534D
:100B3A00856799804E85689980498569998044902E
:100B4A00001EE0F599803CA23BB340077599FAC2B2
:100B5A003B8017A22CB3400575990F800B90005B60
:100B6A00E0F59990005BE4F0C22C8017856A9980C1
:100B7A0012856599800D856B9980087599FC8003AB
:030B8A00754D00A6
:1035BA00020B21020B26020B2B020B30020B3502E7
:1035CA000B3A020B3F020B44020B49020B51020B4E
:0D35DA0076020B7B020B80020B85020B8A30
:0B0B8D009007D0126AA680031235E723
:03341600020B9511
:100B980022E537255AFFAE5950010E90008C126A93
:100BA800BFE0F538E537255AFFAE5950010E0FBFA3
:100BB80000010E90008C126ABFE0F539853F3BE5D5
:100BC80038B539058538378041E539D39538401D22
:100BD800E539C39538853AF0A4FFAEF0E53B8E04BD
:100BE8008F05FF126A88ED2538F537801DE538C373
:100BF8009539853AF0A4FFAEF0E53B8E048F05FFEA
:100C0800126A88EDF4042538F53722E539D395388A
:100C1800401DE539C39538853AF0A4FFAEF0E53BB1
:100C28008E048F05FF126A88ED2538F537801DE59B
:100C380038C39539853AF0A4FFAEF0E53B8E048FB2
:100C480005FF126A88EDF4042538F53722900092E2
:100C5800E0B40170E56675F00A84FF7E008F37E521
:100C68006675F00A84ADF07C008D3A753F0A7559B7
:100C780005755A24E537C394115005120B9980065F
:100C88009005C1E0F537E537900085F0E56675F029
:100C98000A84FF7E008F37E56675F00A84ADF07C24
:100CA800008D3A753F0A755905755A5AE537C39448
:100CB800115005120B9980069005F7E0F537E537D6
:100CC800900016F022900092E0B4016AE56675F093
:100CD8000A84FF7E008F37E56675F00A84ADF07CE4
:100CE800008D3A753F0A755905755A36E537C3942C
:100CF800115005120B9980069005D3E0F53785371A
:100D08004BE56675F00A84FF7E008F37E56675F05F
:100D18000A84ADF07C008D3A753F0A755905755AFD
:100D280048E537C394115005120B9980069005E5E4
:100D3800E0F53785374C22E55E75F00484FF7E00C8
:100D48008F37E55E75F00484ADF07C008D3A753F11
:100D580004755901755A00E537C3943F5005120BC5
:100D68009980069001CBE0F53785372975280090E2
:100D7800005AE075F020A4FFAEF09000DDE08E048C
:100D88008F05FF126A888D379000C5E0D3955E50B5
:100D980003020E459000E9E0D3955E4010ED900106
:100DA800CC126ACAE0F52B752A00020E429000B4F4
:100DB800E0D3955E4043E5379001CC126ACAE0F56E
:100DC80038E5379001EC126ACAE0F5399000E9E09D
:100DD800F404255EF53A9000B4E0FE9000E9E0F4F2
:100DE800042EF53BE538B539058538378003120CF4
:100DF8001385372B752A008041E5379001EC126A7C
:100E0800CAE0F538E53790020C126ACAE0F5399065
:100E180000B4E0F404255EF53A9000C5E0FE9000C9
:100E2800B4E0F4042EF53BE538B53905853837804C
:100E380003120C1385372B752A00020EEC9000EC78
:100E4800E0D3955E5011E53790024C126ACAE0F57E
:100E58002B752A00020EEC9000B5E0D3955E504346
:100E6800E53790022C126ACAE0F538E53790024C53
:100E7800126ACAE0F5399000B5E0F404255EF53A47
:100E88009000ECE0FE9000B5E0F4042EF53BE53868
:100E9800B539058538378003120C1385372B752A29
:100EA800008041E53790020C126ACAE0F538E53750
:100EB80090022C126ACAE0F5399000C5E0F40425C6
:100EC8005EF53A9000B5E0FE9000C5E0F4042EF51A
:100ED8003BE538B539058538378003120C1385375B
:100EE8002B752A00229000FDE0F53C753F117559DD
:100EF80002755A00AE51AF52E53C75F00FA4FDAC37
:100F0800F0EDD39FEC9E4021E53C8E048F05FF1247
:100F18006A88ED75F010A4FFAEF0E55E75F01184F7
:100F2800FD7C00ED2FF53D800EE55E75F01184FF28
:100F38007E00EF24F0F53D853D37E55E75F01184C0
:100F4800AFF07E008F3A120B9985373EAE51AF5203
:100F58009000FDE075F00FA4FDACF0EDD39FEC9E82
:100F68004028755902755A10853D37120B99853EF0
:100F780038853739AE51AF52E53C8E048F05FF12E4
:100F88006AB38D3A853C3B120C13853729752800C6
:100F9800752B64752A00229000FDE0F53C753F1121
:100FA800755902755A00AE51AF52E53C75F00FA461
:100FB800FDACF0EDD39FEC9E4021E53C8E048F05FF
:100FC800FF126A88ED75F010A4FFAEF0E56075F0C9
:100FD8001184FD7C00ED2FF53D800EE56075F01164
:100FE80084FF7E00EF24F0F53D853D37E56075F020
:100FF8001184AFF07E008F3A120B9985373EAE51BF
:10100800AF529000FDE075F00FA4FDACF0EDD39F5A
:10101800EC9E4028755902755A10853D37120B9978
:10102800853E38853739AE51AF52E53C8E048F0581
:10103800FF126AB38D3A853C3B120C13853729752C
:1010480028009000C7E0B40453E55E75F00484FFFF
:101058007E008F37E55E75F00484ADF07C008D3A34
:10106800753F04755901755A00E537C3943F50051B
:10107800120B9980069001CBE0F537AE28AF29E531
:1010880037126A9874648E048F05FF126A88AE2836
:10109800AF29EF2DFDEE3CFC8C288D29752B64754E
:1010A8002A0022900092E0B40146E56675F00A84B1
:1010B800FF7E008F37E56675F00A84ADF07C008D01
:1010C8003A753F0A755905755A00E537C3941150AA
:1010D80005120B99800690059DE0F537AE2AAF2BD7
:1010E800E5372FFF50010E7464126ADC8E2A8F2BAD
:1010F800900093E0B40146E56775F00A84FF7E002E
:101108008F37E56775F00A84ADF07C008D3A753F3E
:101118000A755905755A6CE537C394115005120BB9
:10112800998006900609E0F537AE2AAF2BE5372FF0
:10113800FF50010E7464126ADC8E2A8F2B9000A275
:10114800E0B40249E569C3944175F00584FF7E0067
:101158008F37E56975F00584ADF07C008D3A753FF1
:1011680005755906755A00E537C394135005120BD7
:1011780099800690069FE0F537AE2AAF2BE5372F0A
:10118800FF50010E7464126ADC8E2A8F2B9000E4E3
:10119800E0B40202800302124AE55E75F01584FF8E
:1011A8007E008F37E55E75F01584ADF07C008D3AD2
:1011B800753F15755903755AF4E537C3940B5005F7
:1011C800120B99800690048BE0F537E53775F0FF30
:1011D800A4FFAEF09000E5E08E048F05FF126A8848
:1011E800ED90007EF0E56575F078A4FFAEF074FF31
:1011F8008E048F05FF126A888C598D5A74028C06EA
:101208008D071200398F37AC59AD5A7404FF126A32
:10121800B38D3A753F04755906755A28E537C39456
:101228001D5005120B9980069006D1E0F537AE2ABD
:10123800AF2BE5372FFF50010E7464126ADC8E2A3B
:101248008F2B900091E0B4025DE56075F064A4FF17
:10125800AEF074081200398E5B8F5C74058E048FB3
:1012680005FF126A888D37AE5BAF5C74058E048FFC
:1012780005FF126AB38D3A753F05755905755ADE33
:10128800E537C394135005120B99800690067DE04C
:10129800F537AE2AAF2BE5372FFF50010E746412D5
:1012A8006ADC8E2A8F2B9000D3E0703C90005AE0C5
:1012B80075F00584FF7E008F3790005AE075F005C1
:1012C80084ADF07C008D3A753F05755905755AC097
:1012D800E537C3941D5005120B998006900669E006
:1012E800F537E537900086F02290009AE0B40117B0
:1012F8009007D3E0252BFFAE2A50010E9000EEE0B8
:10130800126ADC8E2A8F2B900112E0B4011490012E
:1013180013E0A851B8000495525007E55EC3955FE5
:10132800400280129000BCE0252BFFAE2A50010E2F
:101338008E2A8F2B802F90009AE0B40316A22EB32A
:10134800B350109007D6E0C39405A851B80006958D
:1013580052400280109000BCE0252BFFAE2A5001BD
:101368000E8E2A8F2B900094E0B40202800302159F
:101378004D900097E0602FE566D394464028900092
:1013880017E0FEA3E0FF9000D2E075F003A4FDACE7
:10139800F0EFD39DEE9C400E9000F6E0A851B80007
:1013A80005D39552500302154D9000DFE0855EF09D
:1013B800A4FFAEF07405126A9874071200398E59AA
:1013C8008F5A90009EE0A851B80004955250129090
:1013D800009FE075F002A4FDACF0EFC39DEE9C40C9
:1013E8000302154DE55E75F00B84FF7E0090061C28
:1013F800126ABFFEE0FFEE900096E0FEEF8E0088D6
:10140800F0A4FFAEF074648E048F05FF126A888C16
:10141800598D5A90005AE075F018A4FFAEF090006C
:10142800DDE08E048F05FF126A888C068D07900612
:1014380034126ABFAE59AF5AE0126A9874648E04C7
:101448008F05FF126A888C598D5AE564A859B8002F
:1014580077D3955A4072E564C3955AFFE49559FECF
:101468008E598F5A7428BE00039F500C755A2875E0
:101478005900740D90005BF0AE59AF5A900097E098
:10148800126A9874288E048F05FF126A888C598D09
:101498005AAE28AF29740A8E048F05FF126A888D08
:1014A800068C07AC59AD5ACFCECF120003740A8E02
:1014B800048F05FF126A888C598D5AAE28AF2912FD
:1014C8006AE48E288F29807DE564A859B8000495C0
:1014D8005A5072AE59AF5AE564126ADC8E598F5A67
:1014E8007428BE00039F500C755A28755900740D56
:1014F80090005BF0AE59AF5A900097E0126A98746A
:10150800288E048F05FF126A888C598D5AAE28AF31
:1015180029740A8E048F05FF126A888D068C07AC21
:1015280059AD5ACFCECF120003740A8E048F05FF2F
:10153800126A888C598D5AAE28AF29EF2DFDEE3CE2
:10154800FC8C288D29229000F2E0B4026AE55E75D1
:10155800F00884FF7E008F37E55E75F00884ADF0F3
:101568007C008D3A753F08755901755AE0E537C317
:10157800943F5005120B99800690028BE0F5378551
:10158800372D752C00AE2CAF2DAC2AAD2B120003D5
:1015980074648E048F05FF126A888C2C8D2D900040
:1015A8008FE08C068D07126A9874648E048F05FF8D
:1015B800126A888C2C8D2DAE28AF29AC2AAD2B123F
:1015C800000374648E048F05FF126A888C288D29A5
:1015D80090008FE08C068D07126A9874648E048FD1
:1015E80005FF126A888C288D29A20D401DAE51AFC7
:1015F800527405BE00039F5002D20DE560D394CC0F
:101608004008D201741190005BF09000F1E0B40240
:10161800089000F3E0640160028035AE28AF29E548
:101628006A126A9874E78E048F05FF126A888C28FC
:101638008D299000F2E0B40217AE2CAF2DE56A12A6
:101648006A9874E78E048F05FF126A888C2C8D2D9A
:101658009000B1E05402601B9000A8E0A851B800C7
:1016680012D39552400DA20DB3B35007E560C39451
:101678009A40028028AE35AF369000A6E075F00299
:10168800A4FDACF0EF2DFDEE3CFC74022DFD5001E5
:101698000CE560BC0007D39D4003754301856036A7
:1016A800753500E5437003021791900104E0C39576
:1016B800435003021783900114E0C394025076E567
:1016C8006675F00A84FF7E0090058C126ABFE0F50B
:1016D8005A755900AE59AF5A9000A7E0126A98742B
:1016E800648E048F05FF126A888C5B8D5C90010400
:1016F800E004C395438C068D07126A98900104E0B4
:101708008E048F05FF126A888C5B8D5CAE28AF292A
:10171800EF2DFDEE3CFC8C288D299000F2E0B40200
:1017280012AE2CAF2DAA5BAB5CEF2BFBEE3AFA8A1C
:101738002C8B2D8046900104E004C39543854BF023
:10174800A4FFAEF0900104E08E048F05FF126A88B2
:101758008C5B8D5CAE28AF29EF2DFDEE3CFC8C2810
:101768008D299000F2E0B40212AE2CAF2DAA5BAB2B
:101778005CEF2BFBEE3AFA8A2C8B2D054390010483
:10178800E0C3954350037543009000B1E0540160F5
:101798001B9000A5E0A851B80012D39552400DA2A5
:1017A8000DB3B35007E55EC394CC4002802590008A
:1017B800A3E075F003A4FFAEF0E5402FFF50010E43
:1017C80074032FFF50010EE55EBE0007D39F400350
:1017D800754401855E40E54470030218C490010514
:1017E800E0C3954450030218B6900114E0C3940274
:1017F8005076E56675F00A84FF7E0090058C126AC3
:10180800BFE0F55A755900AE59AF5A9000A4E012DE
:101818006A9874648E048F05FF126A888C5B8D5CED
:10182800900105E004C395448C068D07126A9890D0
:101838000105E08E048F05FF126A888C5B8D5CAE13
:1018480028AF29EF2DFDEE3CFC8C288D299000F265
:10185800E0B40212AE2CAF2DAA5BAB5CEF2BFBEE13
:101868003AFA8A2C8B2D8046900105E004C39544F2
:10187800854CF0A4FFAEF0900105E08E048F05FFC3
:10188800126A888C5B8D5CAE28AF29EF2DFDEE3C8B
:10189800FC8C288D299000F2E0B40212AE2CAF2DFA
:1018A800AA5BAB5CEF2BFBEE3AFA8A2C8B2D054436
:1018B800900105E0C395445003754400900107E08A
:1018C8002529FFAE2850010E8E288F299000B6E0FA
:1018D800A828B80004952950099000B6E0F52975A4
:1018E80028009000F2E0B4020D9000B6E0A82CB8F1
:1018F8000006952D400280099000B6E0F52D752C64
:1019080000229000F2E0B401028003021A15A20D31
:10191800B35003021A139000BDE0B40168AE28AFBB
:1019280029AC51AD52120003743C8E048F05FF128E
:101938006A889000CDE0BC00109D400D9000CFE07B
:10194800A828B8000495295002D202AE28AF29ACC5
:1019580051AD52120003743C8E048F05FF126A8841
:101968009000CDE0C3940ABC0015D39D40119000AF
:10197800CFE0C39405A828B80005D3952950028064
:1019880002C2028068AE28AF29AC51AD52120003E2
:1019980074788E048F05FF126A889000CDE0BC0031
:1019A800109D400D9000CFE0A828B800049529505C
:1019B80004D2028038AE28AF29AC51AD52120003D0
:1019C80074788E048F05FF126A889000CDE0C39466
:1019D8000ABC0015D39D40119000CFE0C39405A820
:1019E80028B80005D3952950028002C202A202B38A
:1019F8004019AE28AF299000CEE0126A9874648E20
:101A0800048F05FF126A888C288D298002C202A2E1
:101A180000B34006A201B3B3500990001DE4F0A33F
:101A2800F08024AE28AF297400D39F74019E400C27
:101A380090001DE528F0A3E529F0800B74FF9000C5
:101A48001DF8E4F0E8A3F09000D4E0D39402400C31
:101A58009000BFE07006A20DB3B34002801AAE2812
:101A6800AF297402126A988E288F29AE2CAF2D7474
:101A780002126A988E2C8F2D9000BDE0B4011AAE28
:101A880028AF297402126A988E288F29AE2CAF2DA0
:101A98007402126A988E2C8F2DAE28AF29745E12AC
:101AA8006A98740A8E048F05FF126A888C288D291B
:101AB8009000F2E0B40217AE2CAF2D745E126A9853
:101AC800740A8E048F05FF126A888C2C8D2DAE281F
:101AD800AF297402BE000AD39F40067529027528F3
:101AE80000AE2CAF2D7402BE000AD39F4006752DA0
:101AF80002752C0090001BE528F0A3E529F0229040
:101B0800005AE090038C126ACAE0F541754264906D
:101B1800005AE0FE9000C8E0D39E4037E55E75F0BD
:101B28000884FF7E008F37E55E75F00884ADF07C91
:101B3800008D3A753F08755903755A96E537C39471
:101B48001F5005120B998006900441E0F537853740
:101B5800428035E55E75F00884FF7E008F37E55ECC
:101B680075F00884ADF07C008D3A753F087559030F
:101B7800755AB6E537C3941F5005120B9980069025
:101B88000461E0F537853742229000FEE0F53C75A8
:101B98003F11755904755A00AE51AF52E53C75F0C6
:101BA8000FA4FDACF0EDD39FEC9E4021E53C8E04E4
:101BB8008F05FF126A88ED75F010A4FFAEF0E55EA0
:101BC80075F01184FD7C00ED2FF53D800EE55E7506
:101BD800F01184FF7E00EF24F0F53D853D37E55E8A
:101BE80075F01184AFF07E008F3A120B9985373E5D
:101BF800AE51AF529000FEE075F00FA4FDACF0EDD1
:101C0800D39FEC9E4028755904755A10853D3712AC
:101C18000B99853E38853739AE51AF52E53C8E0475
:101C28008F05FF126AB38D3A853C3B120C1385373A
:101C380041754264229000FEE0F53C753F117559EC
:101C480004755A00AE51AF52E53C75F00FA4FDACD7
:101C5800F0EDD39FEC9E4021E53C8E048F05FF12EA
:101C68006A88ED75F010A4FFAEF0E56075F0118498
:101C7800FD7C00ED2FF53D800EE56075F01184FFC9
:101C88007E00EF24F0F53D853D37E56075F0118461
:101C9800AFF07E008F3A120B9985373EAE51AF52A6
:101CA8009000FEE075F00FA4FDACF0EDD39FEC9E24
:101CB8004028755904755A10853D37120B99853E91
:101CC80038853739AE51AF52E53C8E048F05FF1287
:101CD8006AB38D3A853C3B120C13853741754264D3
:101CE8009000F9E0B4047990005AE0FE9000C8E052
:101CF800D39E4037E55E75F00884FF7E008F37E598
:101D08005E75F00884ADF07C008D3A753F08755912
:101D180003755A96E537C3941F5005120B99800630
:101D2800900441E0F5378537428035E55E75F00867
:101D380084FF7E008F37E55E75F00884ADF07C0087
:101D48008D3A753F08755903755AB6E537C3941F20
:101D58005005120B998006900461E0F537853742EB
:101D680022900092E0B4013BE56675F00A84FF7E9C
:101D7800008F37E56675F00A84ADF07C008D3A7502
:101D88003F0A755905755A12E537C3941150051263
:101D98000B9980069005AFE0F537E5422537C394E7
:101DA80064F542900093E0B4013BE56775F00A845E
:101DB800FF7E008F37E56775F00A84ADF07C008DF3
:101DC8003A753F0A755905755A7EE537C39411501F
:101DD80005120B99800690061BE0F537E54225377A
:101DE800C39464F542E5412542F53490009AE0B485
:101DF80002109007D2E02534FE9000EEE0F4042EA5
:101E0800F5349000F1E0D394014040E56AC394E7CB
:101E1800501D74E7C3956AFE9007D4E08E00F5F074
:101E2800E884FF7E008F37E5342537F534801CE5DC
:101E38006AC394E7FE9007D4E08E00F5F0E884FFCB
:101E48007E008F37E534C39537F534A20D4006E59B
:101E5800412464F534E534D394644009E534C394EB
:101E680064F53480037534009000CAE0C39534509B
:101E7800069000CAE0F53422D200900084E0A85110
:101E8800B8000495525041900084E0A851B800046D
:101E98009552500375340F900084E004A851B8009F
:101EA800049552500375340A900084E02402A85126
:101EB800B8000495525005753405C200900084E0BE
:101EC8006006740990005BF0C23E7E017F009000BE
:101ED800D0E0126A989000DFE08E048F05FF126A46
:101EE80088E55EBC0017D39D40139000D9E0B4028A
:101EF80004D23E8002C200740A90005BF09000D1C8
:101F0800E0C3956650159000E3E0A851B800049529
:101F1800525002C200740B90005BF0E566C39464F3
:101F2800501D900129E0600D900129E0A851B800EA
:101F380006955240028008C200740B90005BF0A224
:101F4800004003753405900112E0B40114900113A8
:101F5800E0A851B8000495525007E55EC3955F406C
:101F68000280089000BBE0F534803A90009AE0B413
:101F78000306A22EB3B34002802B9007D6E0C39489
:101F880005A851B800049552500C9000BBE0F534F8
:101F9800740C90005BF09007D6E0A851B800049547
:101FA800525002C20085346B90008CE02534FE90BC
:101FB800005AE075F01E84FC7F00EE2CF534229068
:101FC800005AE075F00584FF7E008F3790005AE0D4
:101FD80075F00584ADF07C008D3A753F05755903A1
:101FE800755AD69000DDE01475F00584FF7E00E593
:101FF80037BE00039F5005120B99800BE5379004FC
:1020080062126ACAE0F537E5379007D5F09007D530
:10201800E0FE9000CCE0C39E50089000CCE0900712
:10202800D5F022E56675F00A84FF7E0090058C12D3
:102038006ABFE0F546E546D394644010E546C3948C
:102048006475F00F84FF7E008F468003754600900C
:1020580000AFE02546F546229007C6E0FEA3E0FF64
:102068007404120039E55E126A98740F8E048F05A5
:10207800FF126A889007C4ECF0A3EDF09000A2E08C
:10208800B40262E569C3944175F00584FF7E008F50
:1020980037E56975F00584ADF07C008D3A753F052C
:1020A800755906755A14E537C394175005120B99DC
:1020B80080069006B3E0F5379007C4E0FEA3E0FF82
:1020C800740A8E048F05FF126A88E5378C068D071F
:1020D800126A98740A8E048F05FF126A889007C4E2
:1020E800ECF0A3EDF09007C4E0FEA3E0FF9007CA70
:1020F800E0FCA3E0FDEDD39FEC9E400F9007CAE003
:10210800F8A3E09007C4C8F0A3C8F0229006D3E073
:10211800903419F8282873804C85527280479000B3
:10212800DFE0855EF0A4FFAEF074081200398F720C
:102138008033856072802E856672802985677280FB
:1021480024856872801F856972801A856A72801575
:102158008565728010856472800B856B728006902D
:05216800001EE0F5720D
:1034190002211F02212102212602213A02213F0213
:10342900214402214902214E02215302215802213D
:073439005D02216202216720
:10216D009006D4E0FE9006D5E0D39E404B9006D36A
:10217D00E0B404189006D5E0C395725002D22F90AA
:10218D0006D4E0D395724002C22F802A9006D4E087
:10219D00C3957250099006D5E0D395725002800216
:1021AD00D22F9006D4E0D3957250099006D5E0C396
:1021BD0095725002C22F802A9006D4E0D3957240BA
:1021CD00099006D5E0C3957240028002C22F900699
:1021DD00D4E0C3957240099006D5E0D395724002C4
:1021ED00D22F229006D7E0903440F8282873804CE7
:1021FD0085527280479000DFE0855EF0A4FFAEF05F
:10220D0074081200398F728033856072802E856656
:10221D007280298567728024856872801F85697236
:10222D00801A856A7280158565728010856472804A
:0C223D000B856B72800690001EE0F572AD
:103440000221FB0221FD02220202221602221B029D
:10345000222002222502222A02222F0222340222C4
:073460003902223E02224363
:102249009006D8E0FE9006D9E0D39E405F9006D76D
:10225900E0B404189006D9E0C395725002D23090C8
:1022690006D8E0D395724002C230803E9006D8E08D
:10227900C3957250099006D9E0D395725002800235
:10228900D2309006D8E0D3957250099006D9E0C3B0
:1022990095725002C2309006D7E0B401099000EB64
:1022A900E0D3956050028002C230802A9006D8E0BF
:1022B900D3957240099006D9E0C395724002800215
:1022C900C2309006D8E0C3957240099006D9E0D390
:1022D90095724002D230229006DBE0903467F828EC
:1022E9002873804C85527280479000DFE0855EF04C
:1022F900A4FFAEF074081200398F728033856072C2
:10230900802E85667280298567728024856872802F
:102319001F856972801A856A7280158565728010B9
:10232900856472800B856B72800690001EE0F572E1
:103467000222EB0222ED0222F202230602230B02C2
:10347700231002231502231A02231F0223240223E7
:073487002902232E0223336A
:102339009006DCE0FE9006DDE0D39E404B9006DB84
:10234900E0B404189006DDE0C395725002D23190D2
:1023590006DCE0D395724002C231802A9006DCE0A7
:10236900C3957250099006DDE0D395725002800240
:10237900D2319006DCE0D3957250099006DDE0C3B6
:1023890095725002C231802A9006DCE0D3957240E2
:10239900099006DDE0C3957240028002C2319006C1
:1023A900DCE0C3957240099006DDE0D395724002E6
:1023B900D231229006DFE090348EF8282873804CC1
:1023C90085527280479000DFE0855EF0A4FFAEF091
:1023D90074081200398F728033856072802E856689
:1023E9007280298567728024856872801F85697269
:1023F900801A856A7280158565728010856472807D
:0C2409000B856B72800690001EE0F572DF
:10348E000223C70223C90223CE0223E20223E7024C
:10349E0023EC0223F10223F60223FB022400022472
:0734AE000502240A02240FAD
:102415009006E0E0FE9006E1E0D39E404B9006DF9B
:10242500E0B404189006E1E0C395725002D23290F0
:1024350006E0E0D395724002C232802A9006E0E0C1
:10244500C3957250099006E1E0D39572500280025F
:10245500D2329006E0E0D3957250099006E1E0C3D0
:1024650095725002C232802A9006E0E0D395724000
:10247500099006E1E0C3957240028002C2329006DF
:10248500E0E0C3957240099006E1E0D39572400201
:10249500D232229006E3E09034B5F8282873804CB8
:1024A50085527280479000DFE0855EF0A4FFAEF0B4
:1024B50074081200398F728033856072802E8566AC
:1024C5007280298567728024856872801F8569728C
:1024D500801A856A728015856572801085647280A0
:0C24E5000B856B72800690001EE0F57203
:1034B5000224A30224A50224AA0224BE0224C302D4
:1034C50024C80224CD0224D20224D70224DC0224FB
:0734D500E10224E60224EBF2
:1024F1009006E4E0FE9006E5E0D39E404B9006E3B3
:10250100E0B404189006E5E0C395725002D233900E
:1025110006E4E0D395724002C233802A9006E4E0DB
:10252100C3957250099006E5E0D39572500280027E
:10253100D2339006E4E0D3957250099006E5E0C3EA
:1025410095725002C233802A9006E4E0D39572401E
:10255100099006E5E0C3957240028002C2339006FD
:10256100E4E0C3957240099006E5E0D3957240021C
:10257100D233229006E7E09034DCF8282873804CAF
:1025810085527280479000DFE0855EF0A4FFAEF0D7
:1025910074081200398F728033856072802E8566CF
:1025A1007280298567728024856872801F856972AF
:1025B100801A856A728015856572801085647280C3
:0C25C1000B856B72800690001EE0F57226
:1034DC0002257F02258102258602259A02259F025C
:1034EC0025A40225A90225AE0225B30225B8022582
:0734FC00BD0225C20225C735
:1025CD009006E8E0FE9006E9E0D39E404B9006E7CA
:1025DD00E0B404189006E9E0C395725002D234902D
:1025ED0006E8E0D395724002C234802A9006E8E0F6
:1025FD00C3957250099006E9E0D39572500280029E
:10260D00D2349006E8E0D3957250099006E9E0C304
:10261D0095725002C234802A9006E8E0D39572403C
:10262D00099006E9E0C3957240028002C23490061B
:10263D00E8E0C3957240099006E9E0D39572400237
:10264D00D234229006EBE0903503F8282873804CA5
:10265D0085527280479000DFE0855EF0A4FFAEF0FA
:10266D0074081200398F728033856072802E8566F2
:10267D007280298567728024856872801F856972D2
:10268D00801A856A728015856572801085647280E6
:0C269D000B856B72800690001EE0F57249
:1035030002265B02265D02266202267602267B02E3
:10351300268002268502268A02268F022694022608
:073523009902269E0226A377
:1026A9009006ECE0FE9006EDE0D39E404B9006EBE1
:1026B900E0B404189006EDE0C395725002D235904B
:1026C90006ECE0D395724002C235802A9006ECE010
:1026D900C3957250099006EDE0D3957250028002BD
:1026E900D2359006ECE0D3957250099006EDE0C31F
:1026F90095725002C235802A9006ECE0D39572405B
:10270900099006EDE0C3957240028002C235900639
:10271900ECE0C3957240099006EDE0D39572400252
:10272900D235229006EFE090352AF8282873804C9C
:1027390085527280479000DFE0855EF0A4FFAEF01D
:1027490074081200398F728033856072802E856615
:102759007280298567728024856872801F856972F5
:10276900801A856A72801585657280108564728009
:0C2779000B856B72800690001EE0F5726C
:10352A0002273702273902273E022752022757026B
:10353A00275C02276102276602276B02277002278F
:07354A007502277A02277FBA
:102785009006F0E0FE9006F1E0D39E404B9006EFF8
:10279500E0B404189006F1E0C395725002D2369069
:1027A50006F0E0D395724002C236802A9006F0E02A
:1027B500C3957250099006F1E0D3957250028002DC
:1027C500D2369006F0E0D3957250099006F1E0C339
:1027D50095725002C236802A9006F0E0D395724079
:1027E500099006F1E0C3957240028002C236900658
:1027F500F0E0C3957240099006F1E0D3957240026E
:10280500D236229006F3E0903551F8282873804C93
:1028150085527280479000DFE0855EF0A4FFAEF040
:1028250074081200398F728033856072802E856638
:102835007280298567728024856872801F85697218
:10284500801A856A7280158565728010856472802C
:0C2855000B856B72800690001EE0F5728F
:1035510002281302281502281A02282E02283302F3
:10356100283802283D02284202284702284C022816
:073571005102285602285BFD
:102861009006F4E0FE9006F5E0D39E404B9006F30F
:10287100E0B404189006F5E0C395725002D2379087
:1028810006F4E0D395724002C237802A9006F4E044
:10289100C3957250099006F5E0D3957250028002FB
:1028A100D2379006F4E0D3957250099006F5E0C353
:1028B10095725002C237802A9006F4E0D395724097
:1028C100099006F5E0C3957240028002C237900676
:1028D100F4E0C3957240099006F5E0D39572400289
:1028E100D237229006F7E0903578F8282873804C8B
:1028F10085527280479000DFE0855EF0A4FFAEF064
:1029010074081200398F728033856072802E85665B
:102911007280298567728024856872801F8569723B
:10292100801A856A7280158565728010856472804F
:0C2931000B856B72800690001EE0F572B2
:103578000228EF0228F10228F602290A02290F027E
:10358800291402291902291E02292302292802299D
:073598002D02293202293740
:10293D009006F8E0FE9006F9E0D39E404B9006F726
:10294D00E0B404189006F9E0C395725002D23890A5
:10295D0006F8E0D395724002C238802A9006F8E05E
:10296D00C3957250099006F9E0D39572500280021A
:10297D00D2389006F8E0D3957250099006F9E0C36D
:10298D0095725002C238802A9006F8E0D3957240B5
:10299D00099006F9E0C3957240028002C238900694
:1029AD00F8E0C3957240099006F9E0D395724002A4
:1029BD00D23822AE2EAF2F74F5D39F74019E4008EE
:1029CD00782E126AEC022ADA752F01752E00AE519F
:1029DD00AF52E546BE000DD39F40099000C1E0D334
:1029ED00954740028023754700E546C39552F57221
:1029FD009000C4E0D395454008E5452572F5458026
:102A0D00069000C4E0F5458002054790009DE0D397
:102A1D009560401CE55EC3955F4015AE51AF52E524
:102A2D0046BE00039F50099000C2E0D39548400276
:102A3D00806E9007D9E0A851B800049552500375E7
:102A4D004A009007D9E0A851B8000BD39552400623
:102A5D00E5529007D9F0E54A7041E552C39546F528
:102A6D0072E572D3940540037572059000C3E0C3FF
:102A7D0095455007E572C3954540028009E545C36C
:102A8D009572F54580069000C3E0F5459000C3E0D2
:102A9D00D3954540069000C3E0F54575480080028A
:102AAD000548E54A701690009DE0C39560500DE510
:102ABD00462405A851B8000695524002800F90009B
:102ACD00B0E0F545754A0174789007D9F022AE2E25
:102ADD00AF2F74E9D39F74039E4008782E126AECD1
:102AED00022C79752F01752E00754532A239402AB9
:102AFD007545199000B0E075F002A4FFAEF0E54702
:102B0D00BE0006D39F4002D2390547754A0374783B
:102B1D009007D9F0754900022C68AE51AF52E546C9
:102B2D006F4E7003022C68E546BE000DD39F400921
:102B3D009000C1E0D395474002800F754700E54AEC
:102B4D00C394035003754519800DE546C39552F5A1
:102B5D0072E5472572F54790009DE0D39560400ED4
:102B6D009007D9E0A851B80007D395524002800CC8
:102B7D0005499000B0E0B54903754A00E54AB40334
:102B8D0006A20DB3B34002800A0549E549B43C03E2
:102B9D00754A02E54AB402299007D9E0A851B80058
:102BAD000ED395524009E5529007D9F07549009022
:102BBD00009DE0C39560500975490074789007D960
:102BCD00F0E54A705A90009DE0D39560401CE55E9B
:102BDD00C3955F4015AE51AF52E546BE00039F5001
:102BED00099000C2E0D395484002800875480075F1
:102BFD00454B8028E552C39546F572E572D3940591
:102C0D00400375720590009DE0D395604008E5483E
:102C1D002572F5488006E5482406F548754900E516
:102C2D004A701690009DE0C39560500DE546240551
:102C3D00A851B80006955240028003754A01E54A35
:102C4D00B4011875451905499000B0E0B5490675F0
:102C5D004A0275490074789007D9F0E54575F00A78
:102C6D00A4FFAEF09007CEEEF0A3EFF022E56E904C
:102C7D00359FF8282873900095E07003022E289058
:102C8D0000CBE0B401028003022D78900058E0B52E
:102C9D005D028003022D757E017F00E5BE126A98EC
:102CAD00E5BD2FFF50010E8E598F5A7410126A9880
:102CBD00900083E08E048F05FF126A889007DAEC8E
:102CCD00F0A3EDF0E56A60089000F1E064026002A7
:102CDD0080269000F3E0B4011F9007DAE0FEA3E038
:102CED00FF74E7126A98E56A8E048F05FF126A88F1
:102CFD009007DAECF0A3EDF0900095E0B402279088
:102D0D0007DCE0FEA3E0FF9007DAE0FCA3E0FDEFB7
:102D1D002DFDEE3CFC74018C068D071200399007D9
:102D2D00DAEEF0A3EFF09007DAE0FEA3E0FF9007F4
:102D3D00DCE0FCA3E0FDEDD39FEC9E4004D23C8093
:102D4D0002B23C9007DAE0F8A3E09007DCC8F0A3EC
:102D5D00C8F09000C7E064016006A23CB3B3400226
:102D6D0080069007DBE0F55E022E26D23C7E017FC9
:102D7D0000E5BE126A98E5BD2FFF50010E8E598FEA
:102D8D005A7410126A98900083E08E048F05FF121A
:102D9D006A889007DAECF0A3EDF0E56A6008900020
:102DAD00F1E06402600280269000F3E0B4011F9010
:102DBD0007DAE0FEA3E0FF74E7126A98E56A8E0475
:102DCD008F05FF126A889007DAECF0A3EDF0900002
:102DDD0095E0B402279007DCE0FEA3E0FF9007DA50
:102DED00E0FCA3E0FDEF2DFDEE3CFC74018C068DA7
:102DFD00071200399007DAEEF0A3EFF09007DAE052
:102E0D00F8A3E09007DCC8F0A3C8F09000C7E06419
:102E1D000160069007DBE0F55E8003755E009000B3
:102E2D0091E07006756E01022C7A75BB180233F3B2
:102E3D00900091E07003022FC97E017F00E5BE1264
:102E4D006A98E5BD2FFF50010E8E598F5A9000D70D
:102E5D00E0B4010F7E0F7FFFAC59AD5A126AE48EBC
:102E6D00598F5A9000FCE0B40245AE59AF5A90000C
:102E7D0027E0FCA3E0FDEDD39FEC9E400A900027D8
:102E8D00E559F0A3E55AF0AE59AF5A900029E0FC90
:102E9D00A3E0FDEFD39DEE9C400A900029E559F08B
:102EAD00A3E55AF0AE59AF5A74041200398F6090F1
:102EBD0000FCE0704CAE59AF5A900027E0FCA3E047
:102ECD00FDEFD39DEE9C4009126AE48E598F5A8016
:102EDD0006755A00755900AE59AF5A7410126A989A
:102EED00900080E08E048F05FF126A888C598D5AF0
:102EFD0074FFBC0009D39D4005855A608003756041
:102F0D00FE9000C7E0B401028003022FC7A20DB3EB
:102F1D00B3500E90009BE0A851B80005D3955250C8
:102F2D0003022FBC90009CE075F019A4FFAEF09049
:102F3D0000DFE08E048F05FF126A889000D8E085CF
:102F4D0060F0A4FFAEF074648D028C038E048F05C7
:102F5D00FF126A88EA2DFDEB3CFC8C598D5AE56A0F
:102F6D00600F9000F1E0B402089000F3E06401609E
:102F7D00028017AE59AF5A74E7126A98E56A8E044B
:102F8D008F05FF126A888C598D5AAE59AF5A90072A
:102F9D00DAE0FCA3E0FDEDD39FEC9E4005855A5E83
:102FAD00800BA23CB340069007DBE0F55E800BA2E0
:102FBD003CB340069007DBE0F55E80037560009042
:102FCD000094E07006756E02022C7A75BB190233FF
:102FDD00F3900094E0700302307EE55DD395504090
:102FED000302307C900025E0FEA3E0FFE564126A49
:102FFD00DC900025EEF0A3EFF07E017F00E5BE1220
:10300D006A98E5BD2FFF50010E8E598F5A90010120
:10301D00E07013740A126A9874518E048F05FF12B2
:10302D006A888D648019AE59AF5A740A126A988FE6
:10303D00048E057E017F95CDCCCD1269868F64E51A
:10304D0064D394644003756464900025E0FEA3E0AE
:10305D00FFE5642FFF50010E900025EEF0A3EFF079
:10306D00900098E0048E048F05FF126A888D6480AD
:10307D00037564329000E4E07006756E03022C7ADD
:10308D0075BB130233F39000E4E0604A7E017F00CC
:10309D00E5BE126A98E5BD2FFF50010E8E598F5A6D
:1030AD0074041200398F659000E6E08565F0A4FD8B
:1030BD00ACF07464FF126A888D659000E5E085655B
:1030CD00F0A4FFAEF074FF8E048F05FF126A88ED39
:1030DD0090007FF08003756500900092E07006759A
:1030ED006E04022C7A75BB170233F3900092E0B494
:1030FD000102800302318C7E017F00E5BE126A98C9
:10310D00E5BD2FFF50010E8E598F5A9007DEE060FE
:10311D00199007DEE01490640412008CE493FC74A3
:10312D000193FDEDC39FEC9E400280069007DEE00B
:10313D0014F09007DEE0C394B3501DAE59AF5A9012
:10314D0007DEE00490640412008CE493FC74019398
:10315D00FDEFC39DEE9C400280069007DEE004F07B
:10316D009007DEE0FE9000B8E08E0088F0A4FFAE80
:10317D00F074648E048F05FF126A888D6680037566
:10318D006600900093E07006756E05022C7A75BB93
:10319D00160233F3900093E0B4010280030232353E
:1031AD007E017F00E5BE126A98E5BD2FFF50010E2E
:1031BD008E598F5A9007DFE060199007DFE0149069
:1031CD00656E12008CE493FC740193FDEDC39FECCE
:1031DD009E400280069007DFE014F09007DFE0C309
:1031ED0094B3501DAE59AF5A9007DFE00490656E51
:1031FD0012008CE493FC740193FDEFC39DEE9C4093
:10320D000280069007DFE004F09007DFE0FE9000FB
:10321D00BEE08E0088F0A4FFAEF074648E048F05BE
:10322D00FF126A888D67800375670075BB1F0233B7
:10323D00F37E017F00E5BE126A98E5BD2FFF5001B8
:10324D000E8E598F5A7409126A9874E68E048F0582
:10325D00FF126A888D6990009AE07006756E0702FC
:10326D002C7A75BB150233F390009AE0700302338C
:10327D008F7E017F00E5BE126A98E5BD2FFF5001DC
:10328D000E8E598F5A74041200398F6890009AE08F
:10329D00B401159000EEE08568F0A4FFAEF0740760
:1032AD00120039EF9007D3F090009AE0B402159018
:1032BD0000EEE08568F0A4FFAEF07407120039EF60
:1032CD009007D2F090009AE0B40302800302338D90
:1032DD009000DBE070389000EEE0601CE568C39470
:1032ED00195002D22EE568D394644002C22E90008C
:1032FD00BAE09007D6F08014E568C394195002D255
:10330D003DE568D394324002C23DC22E80639000E9
:10331D00BAE070349000EEE08568F0A4FFAEF07472
:10332D00FF8E048F05FF126A88ED9007D6F0AE511F
:10333D00AF52741EBE0006D39F4002D22EE560D35D
:10334D0094E54002C22E8029E568C3940A500DAE63
:10335D0051AF52741EBE0004D39F50028002D22E74
:10336D00E560D394E54002C22E9000BAE09007D6F6
:10337D00F09007D6E0C39405500674059007D6F07B
:10338D0080037568009000F1E07006756E08022CE0
:10339D007A75BB1480509000F1E060397E017F009A
:1033AD00E5BE126A98E5BD2FFF50010E8E598F5A5A
:1033BD00EFD39421EE940E4005756AFF8015AE593A
:1033CD00AF5A7410126A9874E38E048F05FF126A57
:1033DD00888D6A8003756A00900095E0600575BB65
:0633ED001A800375BB18F5
:10359F00022C83022E3D022FDE0230930230F802FE
:0B35AF0031A102323E0232750233A34C
:0533F300056ED2EC2282
:096ACA002582F5825002058322A9
:0F008C0025E050020583258250020583F582226C
:106A6700EF2F500205832582F582E5833E2EF583BD
:016A770022FC
:106ADC00CFC39FFF50011E22C3EF9DFFEE9CFE22F1
:086AEC000806B600021806229C
:0D6AA600A3E004F07006120049E004F022A5
:0E003900048007C3CE13CECF13CFD5E0F6223E
:10698600BC000FBE0008ED8FF084FFADF022E4FEE0
:10699600FF22BE000DEF60FE54F0606F20E7030299
:1069A6006A3CEAC0E0EBC0E078017A0075F001EEDF
:1069B60020E710EF25E0FFEE33FE0AC5F023C5F011
:1069C60030E7F0EA5407F9096A7A007B00600108AB
:1069D600C3EC9E40167004ED9F4010ED9FFDEC9EAB
:1069E600FCE5F0CA4ACA03F5F08005E5F003F5F0C8
:1069F600C3EE13FEEF13FFD9D77908CACBCAD8D096
:106A0600EAFEEBFFD0E0FBD0E0FA22EC8FF084FC4C
:106A1600ED54F045F0C48FF084FEEDC454F045F01B
:106A2600C48FF084FDEEC4FE54F02DFFEE540F3CEF
:106A3600FEADF07C0022790078008FF0EC7E082015
:106A4600E70DC3CD33CD33C933C9C833C8DEF084AF
:106A560049F9E5F08FF0BE00E6FD7C00E9FFE8FEAF
:016A6600220D
:0E6A9800F88FF0A4FFE5F0CE88F0A42EFE22C9
:10000300EF8DF0A4F9A8F0EF8CF0A428F8EE8DF0B2
:06001300A428FEE9FF2213
:106A7800600D782B026A82007830D8FED5E0F822C3
:106A8800EEC0E07E00126986EFFDEEFCD0E0FE224B
:0C6AB300EEC0E07E00126986D0E0FE22FA
:03001B0002001EC2
:0300530002005652
:03009B00020071EF
:03000000026AD3BE
:096AD30075817475D000024028A1
:0B6ABF00E5822FF582E5833EF583227F
:0A0049000582D5820215831582227C
:10001E00C0E0C0F0C083C082C0D075D000123F5681
:0B002E00D0D0D082D083D0F0D0E032E0
:10005600C0E0C0F0C083C082C0D075D000123F5946
:10006600D0D0D082D083D0F0D0E032C0E0C0F0C093
:1000760083C082C0D075D000123FDBD0D0D082D0F2
:0600860083D0F0D0E0324F
:00000001FF
